:100000000C945F070C947C070C947C070C947C0781
:100010000C947C070C947C070C947C070C947C0754
:100020000C947C070C947C070C9469310C943B3243
:100030000C943A2C0C947C070C947C070C947C0751
:100040000C947C070C947C070C947C070C947C0724
:100050000C947C070C94C22C0C947C070C947C07A9
:100060000C947C070C947C070C947C070C947C0704
:100070000C947C070C947C070C947C070C947C07F4
:100080000C947C070C947C070C947C070C947C07E4
:100090000C947C070C947C070C947C070C947C07D4
:1000A0000C947C070C947C070C947C078F0C8F0CB1
:1000B000BB0CBB0C230D410D590E590E4C0DE50D1B
:1000C000F60DF60DA832CF32C733CF32C7331B330C
:1000D0003E33C7339533A4334700410043005300F8
:1000E00053435200434150004E554D004C41594539
:1000F00052200068656C6C6F20776F726C64002909
:10010000003A003B003C003D003E003F0040004103
:1001100000420043004C000000000000002B0014CF
:10012000001A000800150017005F00600061001C45
:100130000018000C00120013002A003900040016F9
:1001400000070009000A005C005D005E000B000D66
:10015000000E000F0033453400E1001D001B0006B7
:10016000001900050059005A005B0011001000360C
:10017000003700380028613500E000E300E200AA03
:100180005D2C00620037002E002C00AB5D5000514A
:100190000052004F0029003A003B003C003D003E69
:1001A000003F0040004100420043004C00000000BE
:1001B0000000002B0014001A00090013000A005F61
:1001C00000600061000D000F0018001C0033002AC1
:1001D00000E000040015001600170007005C005D39
:1001E000005E000B00110008000C0012453400E115
:1001F000001D001B0006001900050059005A005B95
:10020000000E00100036003700380028613500E08D
:1002100000E300E200AA5D2C00620037002E002CF3
:1002200000AB5D5000510052004F0029003A003BE6
:10023000003C003D003E003F0040004100420043C2
:10024000004C000000000000002B00340036003796
:100250000013001C005F006000610009000A000636
:100260000015000F002A00E000040012000800182A
:10027000000C005C005D005E0007000B0017001121
:100280000016453800E100330014000D000E001B7D
:100290000059005A005B00050010001A0019001DEB
:1002A0000028613500E000E300E200AA5D2C006256
:1002B0000037002E002C00AB5D5000510052004F63
:1002C0000035021E021F0220022102220223022404
:1002D000022502260227022A000000000000003545
:1002E000021E021F0220022102220201000100015F
:1002F00000230224022502260227024C0001003AB4
:10030000003B003C003D003E000100010001003FB9
:10031000002D022E022F003000310201004000416A
:10032000004200430044000100010001004500328A
:10033000026402010001000100010001000100014E
:10034000000100010001000100010001000100ABFB
:1003500000AA00A900AE0035001E001F00200021E9
:10036000002200230024002500260027002A000088
:10037000000000000035001E001F002000210022A8
:1003800000010001000100230024002500260027B1
:10039000004C004C003A003B003C003D003E000198
:1003A00000010001003F002D002E002F0030003121
:1003B00000010040004100420043004400010001F0
:1003C000000100450032006400010001000100014D
:1003D0000001000100010001002C000100010001EA
:1003E0000001000100AB00AA00A900AE00FD00FE64
:1003F00000FF0001000100010001000100010001F7
:1004000000010001000000000000000100010001E7
:1004100000010001000100010001004A004B00FB47
:1004200000ED00FC00B55D010001000100010001CC
:100430000001000100010001004D004E00EF00EE40
:1004400000F00001000100010001000100010001B5
:10045000000100010001000100F200F300F400F5CA
:10046000000100010001000100010001000100F194
:1004700000010001000100F1000100010001000184
:100480000001003A003B003C003D003E003F0040C0
:10049000004100420043004400450000000000000D
:1004A00000005CC35CC45CC65CC75CC85CC95CCA59
:1004B0005CCB5C010001000100010001004C000167
:1004C00000010001001D5C1E5C135C0100010001C5
:1004D000000A5CA75DA85D01000100010001002B7E
:1004E0005C2A5C265C275C2C5C2D5C010001000111
:1004F000000100BE5CBF5CC15CC05C01000100018A
:1005000000010001000100010001000100010001E3
:1005100000010001000100010000000000000000D7
:10052000002A2B280000000000000000000000004E
:100530000000000029000000002C1E34202122248D
:10054000342627252E362D3738271E1F202122231B
:100550002425263333362E37381F040506070809AD
:100560000A0B0C0D0E0F1011121314151617181973
:100570001A1B1C1D2F3130232D35040506070809D1
:100580000A0B0C0D0E0F1011121314151617181953
:100590001A1B1C1D2F3130354C00000000000000DC
:1005A000000000000000000000000000000000004B
:1005B000000000000000000000000000007E0F00AE
:1005C000D4FFFFFFC70000007800047F3F1F6432A4
:1005D00014643214783C1E1E140A05222325262892
:1005E000292A2C2D2F3032333536383A3B3D3E40C8
:1005F00042434547494A4C4E5051535557595A5C0E
:100600005E6062646668696B6D6F71737577797B24
:100610007D7F81838587898A8C8E90929496989A23
:100620009C9E9FA1A3A5A7A8AAACAEAFB1B3B4B638
:10063000B8B9BBBCBEBFC1C2C3C5C6C7C9CACBCC93
:10064000CDCED0D1D2D2D3D4D5D6D7D7D8D9D9DA66
:10065000DADBDBDBDCDCDCDCDCDDDDDDDDDCDCDCDB
:10066000DCDCDBDBDBDADAD9D9D8D7D7D6D5D4D303
:10067000D2D2D1D0CECDCCCBCAC9C7C6C5C3C2C1D8
:10068000BFBEBCBBB9B8B6B4B3B1AFAEACAAA8A735
:10069000A5A3A19F9E9C9A98969492908E8C8A89ED
:1006A000878583817F7D7B79777573716F6D6B69CA
:1006B00068666462605E5C5A5957555351504E4C9F
:1006C0004A4947454342403E3D3B3A38363533324E
:1006D000302F2D2C2A292826252322FFAA7F55409A
:1006E00000010101010101010101020202020202F5
:1006F00002020203030303030303030404040404C8
:10070000040405050505050606060606070707078E
:100710000708080808090909090A0A0A0B0B0B0C43
:100720000C0C0D0D0D0E0E0E0F0F0F1010111111E0
:100730001212131314141515161617171818191961
:100740001A1A1B1B1C1D1D1E1E1F202021222223C6
:100750002424252626272829292A2B2C2D2D2E2F07
:1007600030313232333435363738393A3B3C3D3E1E
:100770003F404142434445464748494A4C4D4E4F0D
:1007800050515354555658595A5B5D5E5F616264CF
:10079000656668696B6C6D6F7072737577787A7B5C
:1007A0007D7E8082838587888A8C8E8F91939596B3
:1007B000989A9C9EA0A2A3A5A7A9ABADAFB1B3B5D3
:1007C000B7BABCBEC0C2C4C6C9CBCDCFD1D4D6D8AF
:1007D000DBDDDFE2E4E7E9EBEEF0F3F5F8FAFDFF4D
:1007E00000AE00AF00DA0281FFD9F1DB20A4A62E13
:1007F000AF00A0C000A1C800AED580A81FD30040A4
:100800008D14200007087F0807003E5B4F5B3E0009
:100810003E6B4F6B3E001C3E7C3E1C00183C7E3CF9
:1008200018001C577D571C001C5E7F5E1C000018C2
:100830003C180000FFE7C3E7FF0000182418000081
:10084000FFE7DBE7FF0030483A060E00262979294A
:100850002600407F05050700407F05253F005A3CE4
:10086000E73C5A007F3E1C1C0800081C1C3E7F0011
:1008700014227F2214005F5F005F5F0006097F0182
:100880007F00006689956A0060606060600094A2E5
:10089000FFA2940008047E04080010207E201000AF
:1008A00008082A1C0800081C2A0808001E1010103E
:1008B00010000C1E0C1E0C0030383E383000060EA6
:1008C0003E0E060000000000000000005F00000077
:1008D000000700070000147F147F1400242A7F2AD9
:1008E00012002313086462003649562050000008A5
:1008F00007030000001C224100000041221C0000F0
:100900002A1C7F1C2A0008083E080800008070305E
:1009100000000808080808000000606000002010BF
:10092000080402003E5149453E0000427F4000005D
:100930007249494946002141494D33001814127F3C
:1009400010002745454539003C4A494931004121BD
:1009500011090700364949493600464949291E0010
:1009600000001400000000403400000000081422C1
:100970004100141414141400004122140800020150
:10098000590906003E415D594E007C1211127C004F
:100990007F49494936003E41414122007F41414162
:1009A0003E007F49494941007F09090901003E4154
:1009B000415173007F0808087F0000417F4100001B
:1009C0002040413F01007F08142241007F40404009
:1009D00040007F021C027F007F0408107F003E4120
:1009E00041413E007F09090906003E4151215E0058
:1009F0007F091929460026494949320003017F0130
:100A000003003F4040403F001F2040201F003F4068
:100A100038403F00631408146300030478040300A3
:100A20006159494D4300007F4141410002040810D3
:100A30002000004141417F000402010204004040C7
:100A40004040400000030708000020545478400054
:100A50007F2844443800384444442800384444281B
:100A60007F0038545454180000087E09020018A46E
:100A7000A49C78007F080404780000447D400000B6
:100A80002040403D00007F102844000000417F408E
:100A900000007C04780478007C0804047800384462
:100AA00044443800FC182424180018242418FC009E
:100AB0007C080404080048545454240004043F44AF
:100AC00024003C4040207C001C2040201C003C4076
:100AD00030403C004428102844004C9090907C000A
:100AE0004464544C44000008364100000000770084
:100AF00000000041360800000201020402003C260A
:100B000023263C00000000000000404040F0F8F8C0
:100B1000FF38FFF8F83FF8F8FF38FFF8F8F04040EA
:100B20004000000000000080C0C0C0800000C0C0C5
:100B30008000000080C0C000C0C0000080C0C000B5
:100B400000000000C0C0C0C0C000C0C00000000065
:100B50000000000000000000000000000000000095
:100B60000000000000000000000000000000000085
:100B70000000000000000000000000000000000075
:100B8000000000C0F0F8FC3E1E06010000007F419E
:100B900041417F007F4141417F000080C0E07E5B9A
:100BA0004F5BFEC00000C000DCD7DEDEDED7DC001D
:100BB000C000000000000000000000000000000075
:100BC00000000000000000000000494949FFFFFF4D
:100BD000FFE0DFBFBF00BFBFDFE0FFFFFFFF49490E
:100BE0004900000000001F3F6060E0BF1F007F7FE2
:100BF000071E381E077F7F007F7F0E1F3B7160003E
:100C0000000000007F7F0C0C0C007E7E007F7E03C6
:100C100003007F7E03037E7E03037F7E000F3E7012
:100C20003C063C703E0F00327B49493F7E007F7E90
:100C30000303001E3F69696F2600000000000000EA
:100C4000000000030F1F3F3C7870600000007F41F0
:100C500041417F007F4141417F00307B7F783020E0
:100C60002030787F3B0003000F7F0F0F0F7F0F00B6
:100C70000300000000000000000000000000000071
:100C800000000000000000000000010101070F0F3C
:100C90007F0F7F0F0F7E0F0F7F0F7F0F0F07010159
:100CA0000100000000000000000000010100000041
:100CB0000000000000000000000000000000000034
:100CC0000000000000000000000000000000000024
:100CD0000000000000000000000000000000000014
:100CE0000000000000000000000000000000000004
:100CF00000000000000000000000000000000000F4
:100D000000000000000000000000000000000000E3
:100D100000000000000000000000000000000000D3
:100D200000000000000000000000000000000000C3
:100D300000000000000000000000000000000000B3
:100D400000000000200348006100640072006F0092
:100D50006E0020004B006500790062006F006100AA
:100D60007200640000000E036900730068007400E4
:100D70006F00620000000403090409023B00020145
:100D800000A0FA090400000103010100092111017A
:100D90000001224000070581030800010904010049
:100DA000010300000009211101000122B60007051E
:100DB0008203200001120100020000000830FB370E
:100DC0005F02000102000105010902A1018502097B
:100DD00001A10005091901290815002501950875CB
:100DE0000181020501093009311581257F950275C0
:100DF00008810609381581257F950175088106054A
:100E00000C0A38021581257F950175088106C0C03E
:100E100005010980A101850319012AB700150126E2
:100E2000B700950175108100C0050C0901A101856D
:100E30000419012AA002150126A00295017510814E
:100E400000C005010906A1018506050719E029E78B
:100E5000150025019508750181020507190029EF84
:100E60001500250195F07501810205081901290574
:100E7000950575019102950175039101C005010960
:100E800006A101050719E029E71500250195087558
:100E90000181029501750881010507190029FF15D7
:100EA0000026FF009506750881000508190129052F
:100EB000950575019102950175039101C0001124FA
:100EC0001FBECFEFDAE0DEBFCDBF11E0A0E0B1E0A2
:100ED000E6E0FAE602C005900D92A63DB107D9F70B
:100EE00025E0A6EDB1E001C01D92AF37B207E1F7F2
:100EF0000E94931A0C9401350C94000082E008952E
:100F0000EF92FF920F931F93CF93DF930E94492795
:100F1000882309F4C1C060E08CEE90E00E94F925BE
:100F200060910E0270910F02809110029091110257
:100F30000E94D90A61E0805D0E9414250E94EA2A7D
:100F4000C82F60E082E10E94DE246C2F617088EE81
:100F500090E00E94F92561E082E10E94DE24C1FB5D
:100F6000662760F984EE90E00E94F92562E082E154
:100F70000E94DE24C2FB662760F980EE90E00E94AA
:100F8000F9250E945C14C82F63E08AE00E94DE24E9
:100F90008C2F827261E009F460E08EED90E00E9497
:100FA000F9250E94F52461E08C2F817109F460E03D
:100FB0008CED90E00E94F9250E94F52461E08C2FD1
:100FC000847409F460E08AED90E00E94F9250E94A3
:100FD000F524C87861E009F460E088ED90E00E94B3
:100FE000F9250E94F524C0E0EE24E394F12C00E002
:100FF00010E0D4E1DC0F8C2F0E942D199701002EF8
:1010000002C0220F331F0A94E2F78223932341E0A8
:10101000892B09F440E06D2F87E0800F0E94BB25EB
:101020000F5F1F4F0F30110531F7CF5FC530F9F655
:10103000C5E041E062E18C2F0E94BB2541E06BE1FD
:101040008C2F0E94BB25CF5FC83199F7C2E141E0E8
:101050006C2F85E00E94BB2541E06C2F88E10E9447
:10106000BB25CF5FCB3199F741E064E183E10E947A
:10107000BB2541E064E184E10E94BB2541E064E1DD
:1010800085E10E94BB25C0E041E06C2F83E20E9415
:10109000BB25CF5FC830C1F780E0DF91CF911F91B2
:1010A0000F91FF90EF900895CF93DF93D62FC42F29
:1010B0000E94A10F882371F08D2F0E94A10F882319
:1010C00049F080911F030E9465228C2FDF91CF9100
:1010D0000C94C10F8C2FDF91CF910C94E20FCF9322
:1010E000FB018A3A2DE5920739F168F4873A2DE53C
:1010F0009207A1F0883A2DE59207B1F0843C9C4517
:1011000009F09BC07FC08C3A2DE5920709F470C0AE
:10111000D8F1853B9D4509F487C08FC0C281CC239F
:1011200009F48CC080E005C0C281CC2309F486C0DC
:1011300081E00E9472097FC0C281CC23D9F08091E6
:10114000D90181110BC080913703869590E090936F
:10115000200380931F0381E08093D9018091D801FF
:10116000811106C081E08093D80180E10E94652250
:1011700083E027C080911F030E9465221092D8014E
:1011800083E00E94E20F2EC0C281CC2311F1809136
:10119000D90181110BC080913703869590E090931F
:1011A000200380931F0381E08093D9018091D801AF
:1011B000811106C081E08093D8018FE00E946522F2
:1011C00084E00E94C10F46E064E083E00E9454087E
:1011D00032C080911F030E94652284E00E94E20FCA
:1011E0001092D80146E064E083E00E94540826C0D3
:1011F000C28185EECC2319F00E949C0B1CC00E947A
:10120000F20B1CC0C281CC23C9F080911F030E9445
:1012100065220E94552280913703869590E0909335
:10122000200380931F0307C0C281CC2339F083EFD2
:1012300090E00E94D60AC0E001C0C1E08C2FCF919F
:101240000895089581E008950C946F0808950C9412
:1012500026091F93CF93DF9300D000D01F92CDB704
:10126000DEB749835A836B833091DB0189819A8190
:10127000311114C0662359F0222349F00E94B610A0
:10128000182F682F89819A810E945F1003C00E94E5
:101290008A10182F69817A81812F04C00E94B610AC
:1012A00069817A810F900F900F900F900F90DF91CE
:1012B000CF911F910C940018FC01262F4081518181
:1012C0006281738184810C94290981E00895CF9310
:1012D000DF93EC0160E00E945C09BE01DF91CF91D9
:1012E0000C942709CF92DF92EF92FF92C12CD12C60
:1012F0007601C39404C0CC0CDD1CEE1CFF1C8A9547
:10130000D2F78C2D0E945815C701B601FF90EF90BF
:10131000DF90CF900C94410F0C9444190C94421917
:1013200008950E94E90E0E9490092FEF84E39CE04B
:10133000215080409040E1F700C000000C94E82C60
:101340000F931F93CF93DF938C0161E00E945C09A0
:10135000EC01B8010E942409882309F444C0B801B3
:10136000CE010E9473298823F1F1B801CE010E94B9
:1013700087278823C1F1B801CE010E94CF28882396
:1013800091F1B801CE010E945B23882361F1F8013D
:101390008281882309F1CB358DE5D807C1F050F45F
:1013A000C115FCE5DF0781F0CF3DDC45A9F40E94C3
:1013B000F21519C0CC35EDE5DE0761F0CD35DD4520
:1013C00059F40E94301508C00E9491090CC00E9477
:1013D000391502C00E943C15C801DF91CF911F91C1
:1013E0000F910C94220980E0DF91CF911F910F9112
:1013F00008950E941C2C0E943A0B0C942F270E94E7
:101400003D0B0C94222CDF92EF92FF920F931F93CF
:10141000CF93DF93E82FF0E0E75EFA4FD490282FC8
:1014200026952695269530E0F901E754FA4F049168
:10143000877010E0082E02C0159507950A94E2F710
:1014400001701127F901E755FA4FE490F12C082EAD
:1014500002C0F594E7940A94E2F791E0E922FF24B0
:10146000F901E756FA4FC491D0E002C0D595C7956F
:101470008A95E2F7C170DD270115110519F081EE9B
:101480000E949C0BE114F10419F086EE0E949C0B63
:101490008D2D0E943D0CEF2819F086EE0E94F20B74
:1014A000012B19F081EE0E94F20BCD2B51F08CE252
:1014B000DF91CF911F910F91FF90EF90DF900C94EF
:1014C0003D0CDF91CF911F910F91FF90EF90DF9036
:1014D0000895EF92FF920F931F93CF93DF938C01A8
:1014E000F62E8AE0E82EF8018491882309F457C08B
:1014F000813009F042C0E8012196FE0184918130DB
:1015000031F42196FE0184910E943D0C39C0823055
:1015100039F4E8012296FE0184910E949C0B30C0B0
:10152000833039F4E8012296FE0184910E94F20B87
:1015300027C0843029F5E8012296FE01249180E03D
:1015400090E030E0205331092A30310560F4E89E04
:10155000A001E99E500D1124C901840F951F219609
:10156000FE012491EECF009759F0EFE9FFE03197AB
:10157000F1F700C000000197F6CF0E94030AE801CE
:101580008E010F5F1F4F8F2D882309F4ACCFEFE939
:10159000FFE03197F1F700C000008150F5CFDF91F7
:1015A000CF911F910F91FF90EF90089560E00C9400
:1015B000690ACF92DF92EF92FF926C01EE24FF2432
:1015C000C114D104E104F10421F0C701B60120E106
:1015D00001C020E0C72ED82EE92EFF24C114D1046B
:1015E000E104F10419F0285FC701B6016B017C0129
:1015F00054E0F694E794D794C7945A95D1F7C11460
:10160000D104E104F10419F02C5FC701B6016B01AC
:101610007C0142E0F694E794D794C7944A95D1F7B9
:10162000C114D104E104F10419F02E5FC701B60121
:10163000DC01CB01B695A79597958795892B8A2BC9
:101640008B2B09F02F5F822FFF90EF90DF90CF90D0
:10165000089508950C94290B81E008950C942C0BA7
:101660000895CF93C82F0E942A0B8C2F0E942E0B17
:10167000CF91089580E00C94310B0E94DE2A0C94E7
:10168000310B0E94DE2A9091DA01891721F08093B4
:10169000DA010C94310B0895CF93DF93CDB7DEB709
:1016A0002B970FB6F894DEBF0FBECDBF4F83588780
:1016B00069877A878B8761110E947C149E012F5F56
:1016C0003F4F86E0F90111928A95E9F785E0FE0126
:1016D0003796D90101900D928A95E1F789819A8117
:1016E0004C815D81452B31F09F3F31F491E08F3F7C
:1016F00019F403C091E001C090E090FF09C0498156
:101700005A816B817C818D819E810E949D1305C0D1
:10171000C9010E9465098111F2CF2B960FB6F8948A
:10172000DEBF0FBECDBFDF91CF910895FC01808158
:1017300091810E94F8100895CF93882309F450C036
:10174000C82F8CEF8C0F813AD0F46C2F809102015E
:10175000909103010E94572B882349F06C2F8091B0
:101760000201909103010E94E22B0E949E146C2FB3
:1017700080910201909103010E94D72B0CC080E25E
:101780008C0F883058F4C77081E001C0880FCA956B
:10179000EAF70E945F14CF910C949E14EBE5EC0FD6
:1017A000E33040F4F0E0EF59FE4F808190E0CF91BC
:1017B0000C94152BE8E5EC0FE73150F4F0E0EE0F58
:1017C000FF1FED5CFE4F80819181CF910C942B2BFC
:1017D000CD3E30F08C2F0E94181BCF910C94EA1B49
:1017E000CF910895882389F19CEF980F913A40F4A6
:1017F000682F80910201909103010E94E22B0DC09D
:1018000090E2980F983058F4877091E001C0990FDA
:101810008A95EAF7892F0E9465140C949E149BE523
:10182000980F933020F480E090E00C94152B98E50D
:10183000980F973120F480E090E00C942B2B8D3E94
:1018400020F00E94731B0C94EA1B08951F93CF9302
:10185000DF93182FEB010E949C0B209741F08FE93A
:101860009FE00197F1F700C000002197F6CF812F8C
:10187000DF91CF911F910C94F20B893319F060E046
:1018800070E002C060E570E00C94260C882321F023
:101890000E945F140C949E140895882321F00E94E6
:1018A00065140C949E140895CF92DF92EF92FF92EC
:1018B0000F931F93CF93DF937C01D62FC72FFC018B
:1018C0001281058102950F700E9455148823B9F08A
:1018D0001123A9F08C2F807F803421F080E28D0FBE
:1018E000883068F08091220382FD09C082E00E9466
:1018F000FE140E94551491E0D82ED92601C0D12C97
:10190000CC2EC2948FE0C8228C2D90E08C309105B3
:1019100008F0CFC1FC01EA5AFF4F0C945F348C2FC2
:10192000807FCF70882311F0C295C07F112399F07A
:10193000CC2309F4AAC180E28D0F883010F0D111B8
:1019400004C08C2F0E945F1403C08C2F0E946F1460
:101950000E949E149AC18D2F0E94F20BCC2309F491
:10196000A8C180E28D0F883038F1DD2329F18C2F5A
:101970000E94751424C08C2F807FCF70803211F0AC
:10198000C295C07FDD2319F0D130A1F13DC0809117
:10199000220382FF17C0112349F0CC2329F08C2F9A
:1019A0000E945F140E949E1480E070C180E00E943B
:1019B000F20BCC2309F47DC18C2F0E9465140E9488
:1019C0009E1477C1112371F0002341F0013031F4EE
:1019D0000E947F148C2B0E9487146BC10E947F147D
:1019E0008C2B1DC0002319F0013009F462C10E9444
:1019F000941425C0112321F0063008F05AC10EC0FE
:101A0000053008F056C11BC0112361F0002331F0EE
:101A1000F701858180FF39C18F7085838C2F0E94EB
:101A2000460C47C1002359F0D93309F03FC1FFEFFD
:101A300007EE13E0F15000401040E1F735C18C2F64
:101A40000E944D0C36C18C2F86958695837019F0B7
:101A5000813061F02EC1112321F08D2F9C2F9370C6
:101A600002C080E090E00E94152B2BC1112321F0D1
:101A70008D2F9C2F937002C080E090E00E942B2B52
:101A800020C18D2F112319F00E94181B02C00E9443
:101A9000731B0E94EA1B15C18C2F837009F047C08D
:101AA00011110BC12D2F229526952770220F220F81
:101AB0006D2F6F70862F90E0A0E0B0E0022E04C082
:101AC000880F991FAA1FBB1F0A94D2F7D4FF10C01A
:101AD0004FE050E060E070E004C0440F551F661F07
:101AE000771F2A95D2F7409550956095709503C061
:101AF00040E050E0BA01C695C695C3708A019B01CB
:101B0000082B192B2A2B3B2BC901B801C23049F0F5
:101B100058F4C13019F00E94550FCFC00E94430FF6
:101B2000CCC00E94670FC9C00E94410FC6C01123DC
:101B300019F08C2F817001C08695882309F4BDC0EF
:101B40002D2F229526952770220F220F6D2F6F7053
:101B5000862F90E0A0E0B0E0022E04C0880F991F0D
:101B6000AA1FBB1F0A94D2F7D4FF10C04FE050E069
:101B700060E070E004C0440F551F661F771F2A9570
:101B8000D2F7409550956095709503C040E050E0C5
:101B9000BA01C695C695C3708A019B01082B192B03
:101BA0002A2B3B2BC901B801C23049F058F4C1308F
:101BB00019F00E943A1081C00E9428107EC00E9435
:101BC0004C107BC00E947B0F78C0CF70112339F07E
:101BD0008C2F0E94C10F8D2F0E94460C6EC08D2F3E
:101BE0000E944D0C8C2F0E94E20F67C0D23F21F162
:101BF00028F4D03F41F0D13FC1F043C0D33F19F1A9
:101C0000D43F79F03EC0112341F0053008F051C0B7
:101C10008C2F8F710E9407104CC0063008F049C00D
:101C2000F7CF8091220382FF18C0112339F08C2F47
:101C30008F710E94C10F3DC01123C9F38C2F8F718A
:101C40000E94E20F36C0112329F08C2F8F710E9461
:101C5000AC0F2FC00E94870F2CC0112349F0CF7109
:101C60008C2F0E94C10F63E08C2F0E94E31421C0CF
:101C700081E00E94FE140230E0F082E00E94FE1437
:101C800018C0112331F0002391F28D2F0E949C0B7C
:101C900010C0002399F2D93349F41FEF27EE33E047
:101CA000115020403040E1F700C000008D2F0E940D
:101CB000F20B88EF8C0D843020F40E94DE2A0E9403
:101CC000310BDD20C9F00E94511480FD15C0F701D1
:101CD00012820E944B140E94C10FC7010E949D0EE8
:101CE0000E944B14DF91CF911F910F91FF90EF90C5
:101CF000DF90CF900C94E20FDF91CF911F910F9165
:101D0000FF90EF90DF90CF9008950F931F93CF93A4
:101D1000DF93EC01688179818A810E9403118C0133
:101D20000E945E100E942F0FB801CE010E94540C39
:101D3000DF91CF911F910F910895CF93DF93EC0125
:101D4000988189812B813C81232B31F08F3F31F4A5
:101D500081E09F3F19F403C081E001C080E080FD75
:101D60001DC0CE010E94A009811110C00E9455140F
:101D70008823A1F08A81882389F08091220382FD43
:101D80000DC082E0DF91CF910C94FE14CE010E9431
:101D9000850ECE01DF91CF910C946709DF91CF9131
:101DA000089580E090E00E94152B80E090E00E9472
:101DB0002B2B0E947C140E949E140E941B1D0C94CD
:101DC000EA1B80910201909103010E94ED2B0C947B
:101DD000D10E0E946C140C94E10E92959F70963077
:101DE00079F010F4925001C09A50923068F4803F1C
:101DF00069F018F4883E40F409C0843F29F406C015
:101E0000883E20F0813F11F080E0089581E0089540
:101E1000FC01808191810E94F8100E94ED0E0895CE
:101E2000CF93DF9300D000D01F92CDB7DEB70F90D5
:101E30000F900F900F900F90DF91CF910895CF9357
:101E4000DF9300D000D000D0CDB7DEB726960FB616
:101E5000F894DEBF0FBECDBFDF91CF9108950895F6
:101E600008950C94300F0C94310F0E94330F60933F
:101E700012027093130280931402909315020C9433
:101E8000D10E0C94350F0F931F93009112021091F5
:101E900013022091140230911502602B712B822BBA
:101EA000932B1F910F910C94350F0F931F9300915B
:101EB0001202109113022091140230911502602336
:101EC0007123822393231F910F910C94350F0F934D
:101ED0001F9300911202109113022091140230916D
:101EE000150260277127822793271F910F910C9469
:101EF000350F0C94300F0E94790F60930E0270938F
:101F00000F0280931002909311020C94D10E60E0A6
:101F100070E0CB010C947B0F611571058105910573
:101F200029F481E0442361F080E00895DC01CB01D5
:101F300004C0B695A795979587954A95D2F7817075
:101F40000895482F60910E0270910F028091100247
:101F5000909111020C948C0F0F931F9341E050E06D
:101F600060E070E08A019B0104C0000F111F221F76
:101F7000331F8A95D2F7C901B8011F910F910C94B4
:101F80007B0F0F931F9341E050E060E070E004C0CE
:101F9000440F551F661F771F8A95D2F780910E0256
:101FA00090910F02A0911002B09111028A019B0141
:101FB000082B192B2A2B3B2BC901B8011F910F911C
:101FC0000C947B0F0F931F9341E050E060E070E0B2
:101FD00004C0440F551F661F771F8A95D2F740959E
:101FE00050956095709580910E0290910F02A0918E
:101FF0001002B09111028A019B01082319232A23A0
:102000003B23C901B8011F910F910C947B0F0F93D3
:102010001F9341E050E060E070E004C0440F551FA2
:10202000661F771F8A95D2F780910E0290910F025A
:10203000A0911002B09111028A019B010827192773
:102040002A273B27C901B8011F910F910C947B0FE0
:102050000F931F9300910E0210910F022091100216
:1020600030911102602B712B822B932B1F910F91BA
:102070000C947B0F0F931F9300910E0210910F028F
:102080002091100230911102602371238223932347
:102090001F910F910C947B0F0F931F9300910E02D1
:1020A00010910F02209110023091110260277127C8
:1020B000822793271F910F910C947B0F08952FE097
:1020C000929F800D1124E82FE695E695E69587709E
:1020D00051E001C0550F8A95EAF785E0E89FF001CD
:1020E0001124E452FE4F20E030E070E04081CB014B
:1020F000022E02C0969587950A94E2F78170819529
:1021000084278523842781932F5F3F4F2530310516
:1021100069F708952FE0929F800D1124682F66952E
:1021200066956695982F977085E0689FB001112499
:1021300040E050E080E0FB01E40FF51FE452FE4F69
:10214000208130E0092E02C0369527950A94E2F7E7
:1021500021703327042E01C0220F0A94EAF7822B44
:102160004F5F5F4F4530510531F70895BF92CF92D1
:10217000DF92EF92FF920F931F93CF93DF938C0127
:10218000C0900E02D0900F02E0901002F090110269
:102190008091120290911302A0911402B091150245
:1021A000C82AD92AEA2AFB2ACFE1D0E0D701C60102
:1021B0000C2E04C0B695A795979587950A94D2F7EB
:1021C00080FD04C0219790F7B12C07C0BC2EB80148
:1021D0008C2F0E9413180197A9F38B2DDF91CF91BB
:1021E0001F910F91FF90EF90DF90CF90BF900895D7
:1021F000CF93DF93EC010E94B610BE010E9413182A
:10220000DF91CF9108951F93CF93DF93EB019091CE
:10221000DB01992321F0CB010E94F81013C0882321
:1022200049F0CB010E94B610182F682FCE010E94F2
:102230005F1004C0CB010E948A10182FBE01812FAD
:102240000E941318DF91CF911F9108951F93CF9390
:10225000DF93C091160216E080911702C81799F01B
:10226000D0E01C9FF0011D9FF00D1124E85EFD4F92
:102270004081518162817381848195810E941F0F09
:102280002196C770E9CFDF91CF911F9108954091BA
:1022900048025091490260914A0270914B0280912C
:1022A0004C0290914D020C941F0FEF92FF920F93EE
:1022B0001F93CF93DF9380914D0282958F7009F029
:1022C00065C080914A02882309F460C0809116029B
:1022D000F0901702109148020091490260914B0260
:1022E00070914C0291E01F3F09F090E0C091000115
:1022F000D0910101292F96E0E92E8F1509F446C0EF
:102300006115710521F00F3F21F030E003C031E08D
:1023100001C0322F90E030FD36C0E89EF001E99E0A
:10232000F00D1124DF01A85EBD4F11963C9111976D
:10233000301329C03C91311326C012963C9112975C
:10234000311121C013964D915C911497461B570B88
:102350004C175D07C0F480914D028F7080618093AF
:102360004D02E35EFD4F80818F708061808388E441
:1023700092E00E949D0EDF91CF911F910F91FF90EF
:10238000EF900C94261101968770B7CFDF91CF9113
:102390001F910F91FF90EF9008959F92AF92BF927F
:1023A000CF92DF92EF92FF920F931F93CF93DF9321
:1023B000CDB7DEB761970FB6F894DEBF0FBECDBFC5
:1023C0008C0185E0F801DE011D9601900D928A9541
:1023D000E1F7D8011296EC9090914802E091490201
:1023E00020914B0230914C022115310531F0EF3F25
:1023F00031F481E09F3F19F403C081E001C080E027
:10240000B82FB1709B2E80FD47C1D8014C91119619
:102410005C9111971396AD90BC90149788E4C82EE8
:1024200082E0D82EF0904A02B501621B730B209116
:10243000000130910101FF2009F4D9C080914D02C3
:102440006217730708F095C0282F207F09F052C04B
:102450005E1313C0491311C0FE2CE1100EC08F7023
:10246000806180934D020E944711C6010E949D0E1B
:1024700080914D02F80185834DC1AB2831F05F3F5B
:1024800031F481E04F3F19F403C081E001C080E0E6
:1024900080FD03C081E08E2502C080E090E0F82F2F
:1024A000F170FF2E80FF1CC0809116022091170250
:1024B00036E0821709F40BC190E0389FF001399F94
:1024C000F00D1124E85EFD4F6181561306C0608156
:1024D000461303C06281E61203C001968770E9CFFC
:1024E000FE2CEE2009F416C180914D02816080938C
:1024F0004D0254C05E1306C0491304C0E11002C06F
:10250000F80199C0C8010E94080F882361F1EE20EC
:1025100051F120914D02822F82958F7090E00297A9
:1025200074F0809148029091490298878F831986B0
:10253000BB86AA862C87CE0107960E949D0E86E058
:10254000F801A8E4B2E001900D928A95E1F70E94AB
:1025500055110E9447110AC05E1711F1C8010E946F
:10256000080F81112CC0C8010E949D0EFF24F39416
:10257000D1C0282F207F81F77A2DB98AA88A6E2DA5
:1025800089890E94100F88E492E00E949D0E86E0E7
:10259000D6011D928A95E9F70E944711F12CBAC025
:1025A0004913DCCFE110DACFF8018583C8010E941E
:1025B0009D0E86E0D6011D928A95E9F7ABC0EE200C
:1025C00091F220914D02822F82958F7090E00297B8
:1025D0000CF4B5CF80914802909149029A83898387
:1025E0001B82BD82AC822E83CE010196A6CF6217DC
:1025F000730708F044C0FE2CEE2009F4B4CF5E133C
:1026000030C049132EC020914D0220FD21C0822FE1
:1026100082958F70482F50E041155105C9F0F8019F
:1026200025834F30510541F08F5F982F9295907F11
:10263000822F8F70892B8583C8010E949D0E86E0B2
:10264000F801A8E4B2E001900D928A95E1F73CC050
:1026500086E0F801A8E4B2E001900D928A95E1F7D6
:1026600059C0C8010E94080F811169CF80914D02A5
:10267000816080934D02C8010E949D0E4BC07A2D4F
:10268000B98AA88A6E2D89890E94100F86E0D6012A
:102690001D928A95E9F718C0EE2009F464CFC801AD
:1026A0000E94080FF82E882309F45DCF86E0F80118
:1026B000A8E4B2E001900D928A95E1F788E492E0F7
:1026C0000E94960B0E9455110E94471123C04D870E
:1026D0005E878D859E850E94F810292F22952F7088
:1026E000223028F49F7039F0811105C00BC02430CE
:1026F00028F49F7049F4805E883020F0C8010E9461
:102700009D0E9F2CF92C06C0D80115969C91907FA8
:1027100091F7F8CF8F2D61960FB6F894DEBF0FBEFC
:10272000CDBFDF91CF911F910F91FF90EF90DF9080
:10273000CF90BF90AF909F9008951F93CF93DF935A
:10274000CDB7DEB72C970FB6F894DEBF0FBECDBF66
:102750004F83588769877A878B879C87CE01079636
:102760000E94CD118823D1F09F8188852A853B85E1
:10277000232B31F08F3F31F481E09F3F19F403C0E8
:1027800081E001C080E080FD47C04F8158856985A8
:102790007A858B859C850E941F0F3EC086E0FE01D6
:1027A0003796DE01119601900D928A95E1F7FF812F
:1027B000E8856A857B856115710531F0EF3F31F45D
:1027C00081E0FF3F19F403C081E001C080E080FD9B
:1027D00023C02091170230E0C90101968770992724
:1027E0004091160250E084179507F1F1F983EA83CE
:1027F0007D836C8396E0929FD001939FB00D11244E
:10280000A85EBD4FFE01319601900D929A95E1F7B9
:10281000809317020E94261116E080911602909173
:102820001702891771F1189FC0011124885E9D4F0E
:102830000E94CD11882329F1E09116021E9FF0011C
:102840001124E85EFD4F4081518162817381848152
:1028500095810E941F0F8091160290E0019687706B
:10286000992780931602D9CF0E94E90E1092170281
:1028700010921602E8E4F2E086E0DF011D928A95EC
:10288000E9F72C960FB6F894DEBF0FBECDBFDF91EF
:10289000CF911F91089580916E02859585958595BC
:1028A000089580916E028770089590916E029770DE
:1028B00081E009F480E0089580919102089590915B
:1028C0009102892B809391020895809590919102B5
:1028D0008923809391020895109291020895909116
:1028E0009002892B80939002089580959091900298
:1028F0008923809390020895109290020895809108
:102900006F02089508950C9482140C94831490918E
:10291000220392FD08C090916F02981721F08093D6
:102920006F020C948514089580916F02882329F01A
:1029300010926F0280E00C9485140895CF93DF937A
:10294000E0910201F0910301809191028083E09176
:102950000201F0910301908180919002892B808384
:1029600080916F02882381F0E0910201F0910301D0
:102970009081892B808380910201909103010E94B4
:10298000412B81110E949414C0910201D091030146
:1029900040E250E06EE472E0CE010E94AC34892B3C
:1029A00069F080E2FE01AEE4B2E001900D928A95FA
:1029B000E1F7CE01DF91CF910C94ED2ADF91CF9119
:1029C00008950C9482149091220392FD10C098E017
:1029D000899F90011124262B20936E020E94C10F23
:1029E00080916E028595859585950C94E1140C94E3
:1029F000C10F10926E0280E00C94E11420916E02DF
:102A00008095822380936E02982F977099F430E01E
:102A1000482F082E000C550B2417350759F09091BC
:102A2000220392FD07C08595859585950E94E20F4A
:102A30000C94F91408959091220392FB222720F917
:102A4000281769F080FB92F990932203809121036B
:102A5000909122030E946E1582E00C94FE1408955A
:102A60008091220382FB882780F991E089270C94CA
:102A70001B1581E00C941B1580E00C941B156FEF67
:102A80007FEF80E090E00C94EB3480E090E00E94D7
:102A9000C73421E0893E9E4F09F020E0822F08953F
:102AA00082E090E00C94B93483E090E00C94B93467
:102AB000682F83E090E00C94CD34CF9384E090E0D5
:102AC0000E94B934C82F82E290E00E94B9342C2FC2
:102AD00030E0A901582BCA01CF910895CF93C92F97
:102AE000682F84E090E00E94CD346C2F82E290E069
:102AF000CF910C94CD34AB01BC018FE090E00C94ED
:102B0000DF34AB01BC0183E190E00C94DF3460E082
:102B100070E0CB010C94811560E070E0CB010E9465
:102B20007B150C94871569EE7EEF80E090E00E94A3
:102B3000EB3460E082E090E00E94CD3460E083E01E
:102B400090E00E94CD341092120210921302109263
:102B500014021092150260E084E090E00E94CD34EF
:102B600060E082E290E00E94CD3460E085E090E099
:102B70000E94CD3460E086E090E00E94CD346FEF9B
:102B800087E090E00E94CD3440E050E0BA0188E058
:102B900090E00E94DF3460E08DE090E00E94CD3450
:102BA00040E050E0BA0188E190E00E94DF3460E04C
:102BB00087E190E00E94CD3440E050E0BA018CE122
:102BC00090E00E94DF3460E070E080E290E00E94DC
:102BD000EB3440E050E0BA0188E190E00E94DF343D
:102BE0000C948C150C949315682F8EE090E00C9447
:102BF000CD340E94A72C6093A0027093A102809311
:102C0000A2029093A30260939C0270939D02809312
:102C10009E0290939F02089585B7806885BF85B70F
:102C2000806885BF089581E008950C941316089577
:102C30000C9417160C9417160C941A160C9417165D
:102C40000C941E160C9417160E940C168FEE98E129
:102C50000E94D42A0E9422160C9420160E94181654
:102C60000C9417160E9409190C94300B0E94922C98
:102C70000E94EC190E94321680E00E9494240E9467
:102C80007A220C941C165F926F927F928F929F9281
:102C9000AF92BF92CF92DF92EF92FF920F931F936A
:102CA000CF93DF93CDB7DEB72A970FB6F894DEBF88
:102CB0000FBECDBF0E94011AC82E81110E94F915C6
:102CC00032E9832E32E0932E00E010E0502E802F68
:102CD0000E942D195C01F401619071904F016826EA
:102CE000792661147104B1F40F5F1F4F053011058F
:102CF00069F78FEF89838A831B820E949B2C8160F6
:102D0000782F9D838C8349815A816B818D810E94AC
:102D10004C0B3AC08091A40281FD0E943619D12C3F
:102D2000EE24E394F12CC3018E219F21892B29F1FC
:102D30000E9415168823A9F0DE825F82AE20BF2094
:102D400081E0AB2809F480E088870E949B2C816099
:102D5000782F9A8789874E815F8168858A850E944E
:102D60004C0B000F111FF801EE56FD4F8081918131
:102D7000E826F926F182E08207C0D394EE0CFF1C0E
:102D8000FFE0DF12D0CFB0CF81E0C11001C080E002
:102D90002A960FB6F894DEBF0FBECDBFDF91CF915C
:102DA0001F910F91FF90EF90DF90CF90BF90AF9069
:102DB0009F908F907F906F905F900895CF930E9427
:102DC0004316C82F0E94AD220E944B27C1110E94BA
:102DD0000B260E94081CCF910C94410BCF93DF93DC
:102DE0000E941818EC01811521E5920708F045C0F2
:102DF000811530E5930708F094C0883E910528F5C9
:102E0000803E910508F0F8C0883A910570F4853A43
:102E1000910508F07CC08130910509F475C008F473
:102E2000E8C0049708F0E8C0E4C08F3B910508F0C3
:102E3000E0C0C85AD0E0CC0FDD1FCC59DE4F09905E
:102E4000D881C02DCE019464D8C0811540E294078A
:102E500058F4811551E0950708F0CEC08D3E9105DC
:102E600008F4C7C09065C9C0C11580E4D80708F44C
:102E7000C0C0DF70CE01906AC0C0811525E5920701
:102E8000A8F4811534E5930708F095C0811543E552
:102E9000940708F07BC0811552E5950708F061C0E2
:102EA000D82FCC27CE01816F906AA7C0C11589E5C4
:102EB000D807A0F4C11528E5D20708F082C0C115D3
:102EC00036E5D30708F095C08C2F0E94AC188F719F
:102ED00090E0D82FCC27CE0190628FC0C1154AE573
:102EE000D40708F474C0CE0190568115904208F0C2
:102EF00080C08D2F8F710E94AC18DD27D0628F713A
:102F0000AE01582BCA0179C081E090E076C0C55A65
:102F1000D0E0CE56DE4F8881C82FD0E0CE0190643D
:102F20006CC074E0969587957A95E1F7282F237009
:102F30003C2F337081E090E002C0880F991F3A95D2
:102F4000E2F79C68AC01522B9A019C2F9F709695DA
:102F5000969550E2959FE0011124C9018C2B9D2B81
:102F60004CC08370992721E030E002C0220F331F4C
:102F70008A95E2F79C2F9695969580E2989FE001BE
:102F80001124C22BD32BCE019C6837C083709927A4
:102F900021E030E002C0220F331F8A95E2F79C2F18
:102FA0009695969540E2949FE0011124C22BD32B75
:102FB000CE019A6822C0D82FCC27CE01846F906AA8
:102FC0001CC0DC2FCC27CE01806F906A16C08C2FDE
:102FD0008F700E94AC1894E0D695C7959A95E1F74A
:102FE000CF70D0E0DC2FCC27D0699E01282BC901FF
:102FF00004C080E090E001C0CE01DF91CF91089540
:103000002BE4829FC0011124FC012FE0729FE00D90
:10301000F11D1124E60FF11DEE0FFF1FE150FF4FD0
:103020008591949108950E9400180E94EE160895CB
:103030008238910569F1B0F48133910509F46DC0CE
:1030400048F48932910509F463C08A32910509F484
:1030500069C008958533910509F455C089339105F8
:10306000B9F00895833E910569F138F4803E9105E9
:10307000B1F0823E910509F10895863E9105A9F1CE
:10308000873E9105B9F1843E910509F064C023C0E3
:103090002091210320FD4FC021FD4DC00895809156
:1030A000210380FD44C08091220380FF44C08091B1
:1030B000210384FD42C083EE4DC08091210382FF35
:1030C00038C0F5CF8091210382FD33C08091220367
:1030D00080FD31C0ECCF8091220381FF32C080910E
:1030E000210384FD2AC087EE35C08091210383FF30
:1030F00026C0F5CF8091210383FD21C0809122035A
:1031000081FD1FC0ECCF8091210385FD1CC01DC037
:103110008091210385FD19C016C08091210386FD91
:1031200016C017C08091210386FD13C010C089E32B
:1031300011C082EE0FC080EE0DC080E00BC086EEA5
:1031400009C084EE07C089E205C085E303C08AE2B6
:1031500001C081E390E008959091210392FF0DC09A
:10316000282F2871283019F4877F846006C0282F03
:103170002471243011F48B7F886093FF0DC0282FB9
:103180002871283119F4877E846106C0282F2471A4
:10319000243111F48B7E88612091220320FF0DC021
:1031A000382F3871383019F4877F816006C0382F86
:1031B0003171313011F48E7F886021FF0DC0282FCE
:1031C0002871283119F4877E816106C0282F21716A
:1031D000213111F48E7E886194FD877E089580E010
:1031E00008950C943F150E94011A8FE39CE9019702
:1031F000F1F700C000000E94011A80E00E942D1922
:1032000080FF04C00E94F1180C94E82C08950C94DF
:10321000F3180E944515811102C00E94F2150E9408
:1032200050158093A4020E945D1590932203809311
:1032300021030E9407190E945415682F70E080E056
:1032400090E00E94410F60910E0270910F028091F8
:103250001002909111020C94790FE82FF0E0EE0F1C
:10326000FF1FE35DFC4F808191810895089580EAFE
:103270008A95F1F7089500C008950C9437190895C0
:103280000C943F190C9440190C942109F894E82FE0
:10329000E295EF70F0E031A1282F2F7081E090E0EF
:1032A00001C0880F2A95EAF7982F9095932391A350
:1032B00092A1892B82A3789408950F931F93CF93A3
:1032C000DF93C4EAD1E089918F3F11F00E94461943
:1032D00081E0C93AD807B9F7C5E9D1E004EA11E0BD
:1032E00089918F3F11F00E9446190C171D07C1F7F5
:1032F000DF91CF911F910F910895BF92CF92DF92EE
:10330000EF92FF920F931F93CF93DF938C01C62F01
:10331000D0E0CE018C559E4F6C01FC0190819F3F07
:1033200009F450C0B62EF894E92FE295EF70F0E062
:1033300081A19F7021E030E001C0220F9A95EAF749
:10334000822B81A382A12095282322A378940E9416
:103350003B19E5E9F1E044EA51E021E030E0E12CFD
:10336000F12C61916F3F89F0A62FA295AF70B0E06C
:1033700090968C9190E06F7002C0959587956A95B4
:10338000E2F780FD02C0C90102C080E090E0E82AB7
:10339000F92A220F331F4E175F0719F7F6018081B4
:1033A0008F3F11F00E94461961E0E114F10409F425
:1033B00060E08B2D0E943D19CC0FDD1FC00FD11F87
:1033C000F982E882DF91CF911F910F91FF90EF90EA
:1033D000DF90CF90BF9008950E945D198AE0EDE2E2
:1033E000F3E0DF01982F1D929A95E9F7E3E2F3E00D
:1033F000DF011D928A95E9F785E00E944C1A0C9432
:103400008C09FF920F931F93CF93DF93CDB7DEB755
:103410002A970FB6F894DEBF0FBECDBF8E010F5FA7
:103420001F4F8AE0F80111928A95E9F7F12C6F2D70
:10343000C8010E947D19F394F5E0FF12F8CF4AE02D
:1034400050E0B80183E293E00E94AC34FF24F3948F
:10345000009709F4F12C892B41F08AE0F801A3E2EE
:10346000B3E001900D928A95E1F72F2D45E06DE2D2
:1034700073E083E293E00E944D1A0E948E098F2D23
:103480002A960FB6F894DEBF0FBECDBFDF91CF9165
:103490001F910F91FF9008950895FF920F931F932E
:1034A000CF93DF93F82E092F162FD72FC42F222367
:1034B00049F081E08093A7020E949B2C9093A60282
:1034C0008093A5028091A7028823D9F08091A5025C
:1034D0009091A6020E94B32C059798F0EF2DF02F43
:1034E000A12FBD2F80E090E04C2F50E0841795076E
:1034F00034F4219131912D933D930196F7CF1092A1
:10350000A702DF91CF911F910F91FF9008950E9424
:10351000C12E0E9436160C94CD2E0E94D12E0E94F0
:10352000DE160C94EB2E0E94392C0E94A82E0E94CD
:1035300024160E94871A0E948D1A0E942E16FBCF15
:103540008091AE0280FF06C06091090170E0660FB5
:10355000771F26C081FF04C06091090184E005C087
:1035600082FF07C06091090188E0689FB0011124C3
:1035700017C09091AD029923D1F060910801961780
:1035800088F72091090188E0289F90011124929FDB
:10359000A001939F500D112470E0CA010E942934AC
:1035A0006038710540F46115710519F406C068E0D2
:1035B00070E0862F08958FE7089581E00895809147
:1035C000AE0280FF08C06091050170E075956795B7
:1035D0007595679521C081FF06C06091050170E077
:1035E0007595679519C082FF04C06091050170E070
:1035F00010C09091AC02992399F060910401961744
:10360000A0F780910501899FC001112470E00E94FC
:1036100029346038710540F46115710519F406C04C
:1036200061E070E0862F08958FE7089581E00895A6
:103630008D3E21F40E94A01A819504C08E3E29F48B
:103640000E94A01A8093B20208958F3E21F40E9436
:10365000A01A819504C0803F29F40E94A01A80938B
:10366000B1020895893F19F40E94DF1A05C08A3F0C
:1036700031F40E94DF1A81958093B30208958B3F45
:1036800021F40E94DF1A819504C08C3F29F40E9426
:10369000DF1A8093B40208959FE0980F983078F471
:1036A00021E030E0A90102C0440F551F9A95E2F7CE
:1036B000CA019091B002892B8093B00208958D3F8A
:1036C00021F48091AE0281600BC08E3F21F4809185
:1036D000AE02826005C08F3F29F48091AE02846003
:1036E0008093AE0208958D3E39F49091B20297FF17
:1036F00035C01092B20259C08E3E29F49091B202A8
:103700001916BCF32BC09091B1028F3E29F497FF9C
:1037100025C01092B10249C0803F19F41916CCF3AC
:103720001DC09091B302893F29F41916BCF4109280
:10373000B3023BC08A3F19F497FF10C0F8CF8B3F0C
:1037400039F49091B40297FF09C01092B4022DC0D1
:103750008C3F21F49091B4021916BCF39FE0980FAE
:10376000983080F421E030E0A90102C0440F551FD9
:103770009A95E2F7CA0180959091B00289238093CF
:10378000B00213C08D3F21F48091AE028E7F0BC03A
:103790008E3F21F48091AE028D7F05C08F3F29F4CA
:1037A0008091AE028B7F8093AE028091B102811135
:1037B00006C08091B202811102C01092AD028091C8
:1037C000B302811106C08091B402811102C010922F
:1037D000AC0208950E949B2C2091B102211104C0DB
:1037E0002091B202222321F09093AB028093AA028F
:1037F0002091B302211104C02091B402222321F0B0
:103800009093A9028093A8028FEA92E00C94072B70
:10381000EF92FF920F931F93CF93DF9300D000D0CE
:1038200000D0CDB7DEB786E0EFEAF2E0DE01119618
:1038300001900D928A95E1F7E090B102F090B2020A
:103840000091B3021091B4021092B1021092B20230
:103850001092B3021092B402E11003C0FF2009F4E9
:103860005DC08091AA029091AB020E94B32CAC0182
:103870009091AD02992339F020910A0130E024178C
:10388000350758F04BC020910B018AE0289F90012A
:1038900011242417350718F041C09F3F19F09F5F8E
:1038A0009093AD02EE2061F00E94A01A1E1414F055
:1038B0009FEF01C091E0989F902D11249093B10249
:1038C000FF2061F00E94A01A1F1414F09FEF01C0A6
:1038D00091E0989F902D11249093B2023091B10203
:1038E0003323E1F02091B2022223C1F045EB3403EF
:1038F000C0011124992319F09093B10203C081E013
:103900008093B10235EB2303C0011124992319F0F0
:103910009093B20203C081E08093B202011103C010
:10392000112309F45DC08091A8029091A9020E9420
:10393000B32CAC019091AC02992339F0209106018F
:1039400030E02417350758F04BC0209107018AE07A
:10395000289F900111242417350718F041C09F3F7C
:1039600019F09F5F9093AC02002361F00E94DF1A70
:10397000101614F09FEF01C091E0989F902D112434
:103980009093B302112361F00E94DF1A111614F014
:103990009FEF01C091E0989F902D11249093B40265
:1039A0003091B3023323E1F02091B4022223C1F01D
:1039B00045EB3403C0011124992319F09093B3020D
:1039C00003C081E08093B30235EB2303C0011124CF
:1039D000992319F09093B40203C081E08093B4025C
:1039E0008091B10281110BC08091B202811107C098
:1039F0008091B302811103C08091B40281110E94B1
:103A0000EA1BEB82FC820D831E8386E0FE01319669
:103A1000AFEAB2E001900D928A95E1F726960FB6D3
:103A2000F894DEBF0FBECDBFDF91CF911F910F91F4
:103A3000FF90EF900895EFEAF2E086E0DF011D923B
:103A40008A95E9F71092AD021092AC021092AE0284
:103A50000895EF92FF920F931F93CF93DF938B0103
:103A6000682F11110AC0442329F0E82FF0E0E0523A
:103A7000F94F6491762F862F75C0212F30E0E82F03
:103A8000F0E0442321F0E052F94FE491F0E046E009
:103A9000049FC0011124CFEFD0E0BE010E94153475
:103AA0004BEA4603C001479F900D1124800F911DE2
:103AB000800F911D982F990F890FAE01421B530B58
:103AC0004E9FD0014F9FB00D5E9FB00D11249B2FD4
:103AD000189FA0011124452F55278E01041B150B9B
:103AE0000E9FA0010F9F500D1E9F500D11247E01AF
:103AF000E81AF108E29E8001E39E100DF29E100D7F
:103B00001124212F3327C21BD30BCE9F9001CF9FAF
:103B1000300DDE9F300D112462307105A9F048F49C
:103B20006115710569F061307105C9F48B2F752F2E
:103B30000DC06430710581F058F06630710579F47C
:103B40007E2F8B2F932F0DC0832F7B2F9E2F09C08D
:103B50008E2F7B2F952F05C08E2F732F02C07E2FA7
:103B6000852F692FDF91CF911F910F91FF90EF90DB
:103B7000089541E00E94291D089508950E94B91DED
:103B80000895CF93DF93762FE901682F842F0E9449
:103B9000BE1D798368838A83DF91CF9108958091D8
:103BA0003703282F269530E02115310519F481704F
:103BB000826005C02532310524F0817088648093CD
:103BC0003703089588E090E00C94C134CF92DF92DF
:103BD000EF92FF926B017C010E94CF1DB701A601FD
:103BE00088E090E0FF90EF90DF90CF900C94DF346E
:103BF000E7E3F3E083E0808311828FEF82838383A6
:103C0000148260817181828193810C94E61D809180
:103C1000370380FF02C08695089580E00895909153
:103C20003B03933018F49F5F90933B03882351F03C
:103C300060913703709138038091390390913A0372
:103C40000C94E61D089581E00C940F1E90913B03A7
:103C5000992319F0915090933B03882351F0609180
:103C60003703709138038091390390913A030C9493
:103C7000E61D089581E00C94261E70E00C942A2421
:103C8000609110018091370380FF0AC080910F017D
:103C900023E0829FC0011124845C9C4F0C943D1E44
:103CA0008091110190911201891780F7E82FF0E0BF
:103CB0009F01220F331FE20FF31FE45CFC4F1182C0
:103CC000108212828F5FF0CF9091370390FF16C061
:103CD0009091110120911201921770F4E92FF0E0F8
:103CE000DF01AA0FBB1FEA0FFB1FE45CFC4F8183BF
:103CF000608342839F5FF0CF0C94401E0895CF9362
:103D0000DF9300D01F92CDB7DEB79091370390FFBD
:103D10000AC09E012F5F3F4F0E94C11D4B816981E8
:103D20008A810E94641E0F900F900F90DF91CF91B7
:103D30000895CF93DF93EC01EC81F0E0E552FA4F68
:103D40004491E7E3F3E0628181810E947F1E8C81D0
:103D50008F5F8C83DF91CF910895CF93DF93EC0138
:103D6000E7E3F3E0438162818C810E947F1E8C81B6
:103D70008F5F8C83DF91CF9108950F931F93CF9323
:103D8000DF9300D01F92CDB7DEB78C018091B502D2
:103D900081110AC09E012F5F3F4F4FEF6FEF0E94CE
:103DA000C11D8A818093B502F8018481813051F070
:103DB00028F0823061F44091B5020AC08091B502CA
:103DC00040E007C06091B50240E080E003C040E001
:103DD00080E060E00E94641EF801848190E001961A
:103DE00063E070E00E94293484830F900F900F905D
:103DF000DF91CF911F910F910895AF92BF92CF9213
:103E0000DF92EF92FF920F931F93CF93DF9300D037
:103E10001F92CDB7DEB7182FF62E042FE22E909109
:103E2000370390FF6DC0E92FE695AE2FB0E0A755A0
:103E3000BE4F8C918093BF029E7F923061F49E01B1
:103E40002F5F3F4F812F0E94C11D4B8169818A8165
:103E50000E94641E43C0823019F400913A033EC0B0
:103E6000863019F41091380339C08930D9F389317B
:103E7000A9F5E9518E2F8170D82EE695F0E0E55234
:103E8000F94FA590B490C12CBB2460911301C616C4
:103E900018F52C2D30E0A29EC001A39E900DB29E7D
:103EA000900D112470E00E941534812FD11002C0B2
:103EB000860F01C0861B90911101290F311DA901A8
:103EC000440F551F240F351F245C3C4F402F6F2D8E
:103ED0000E94C11DC394D9CF0E94401E1093380385
:103EE000F092390300933A03EE2051F060913703CA
:103EF000709138038091390390913A030E94E61D36
:103F00000F900F900F90DF91CF911F910F91FF9025
:103F1000EF90DF90CF90BF90AF900895E7E3F3E08C
:103F20009181282F438162818AE0890F0C94FD1EC4
:103F300081E00C948E1FE7E3F3E09181282F438109
:103F4000628186EF890F0C94FD1E81E00C949B1F0B
:103F5000E7E3F3E0628121E1620F08F46FEF282FBD
:103F6000438181810C94FD1E81E00C94A81FE7E33E
:103F7000F3E0628121E1621B08F460E0282F4381B5
:103F800081810C94FD1E81E00C94B71FE7E3F3E000
:103F9000438121E1420F08F44FEF282F6281818194
:103FA0000C94FD1E81E00C94C61FE7E3F3E043810F
:103FB00021E1421B08F440E0282F628181810C94AA
:103FC000FD1E81E00C94D51F20E00C94FD1EFF9295
:103FD0000F931F93CF93DF93EC01F12C0FEF10E0C1
:103FE00060911301F616F0F4809111012F2D30E04D
:103FF000280F311DC901880F991F280F391F245C14
:104000003C4F70E0C8010E942934962F8C8140916A
:104010003A0360913903F99E800D11240E94C11D5D
:10402000F394DECF0E94401E9A818C8190FF02C0E3
:104030008F5F01C081508C83DF91CF911F910F91D1
:10404000FF900895AF92BF92CF92DF92EF92FF92CE
:104050000F931F93CF93DF93FC01828180FF02C0F7
:104060000FEF01C001E010E04EE0A42E809113019B
:10407000181708F043C080911101C12ED12CE60120
:10408000C80FD11DCE01880F991FC80FD91FC45C5E
:10409000DC4F198218821A8234E0E32EF12CB12C05
:1040A0008091B7028B0D8F302CF06A2D0E9407345F
:1040B000892F05C087FF03C090911301890F082E37
:1040C000000C990BC816D90691F480913A038E9D85
:1040D000A0018F9D500D11245595479555954795F5
:1040E0009E0160913903809138030E94C11DB00E7A
:1040F000F1E0EF1AF108A1F61F5FB8CF0E94401E51
:104100008091B702013031F4811102C08091130116
:10411000815007C090E001966091130170E00E9409
:1041200029348093B702DF91CF911F910F91FF90B7
:10413000EF90DF90CF90BF90AF900895CF93809194
:10414000110190911201891770F4E82FF0E09F019E
:10415000220F331FE20FF31FE45CFC4F1182108229
:1041600012828F5FF0CFC0E060911301C617C0F5D7
:10417000EC2FF0E070E0CF010E9429342091110172
:10418000820F2091B602022E000C330B90E0E21752
:10419000F307CCF020910E01022E000C330B2E17EA
:1041A0003F078CF09C01220F331F820F931F9C014D
:1041B000245C3C4F40913A0360913903809138036D
:1041C0000E94C11D0BC0FC01EE0FFF1F8E0F9F1F31
:1041D000FC01E45CFC4F118210821282CF5FC4CFDD
:1041E0000E94401E20910D018091B602820F8093A3
:1041F000B60290910E01920F90930E0119165CF485
:10420000082E000C990B4091130150E041505109C8
:10421000841795071CF0219520930D01CF910895E7
:104220008F929F92AF92BF92CF92DF92EF92FF92C6
:104230000F931F93CF93DF938C01FC014481C42F14
:10424000D0E09E01DE010E946D349B01AC010E9412
:1042500083346B017C01E0E2F0E0EC1BFD0BA5E593
:10426000B0E09B01AC010E9483344B015C019F01D3
:10427000DF010E9465349B01AC010E948E349B01DA
:10428000AC012C0D3D1D4E1D5F1DC501B4010E94EA
:104290003D34C22FD22F2A3228F4F3E02F9F900111
:1042A00011240DC025E530E02C1B3109C901880F10
:1042B000991F280F391F37FF02C02F5F3F4F3595D9
:1042C0002795C22FC095F12C85E5E82EED1A809137
:1042D0001301F816C8F4F1FC02C08E2D01C08D2F19
:1042E000909111012F2D30E0290F311DA901440FAC
:1042F000551F240F351F245C3C4F4C2F6091390310
:104300000E94C11DF394E3CF0E94401EF8018481F6
:10431000811102C091E003C0803219F49FEF9093A5
:104320000C0190910C01890FF8018483DF91CF91EA
:104330001F910F91FF90EF90DF90CF90BF90AF90C3
:104340009F908F9008950F931F93CF93DF93EC016D
:1043500000E010E080911301282F30E002171307CE
:1043600024F5909111019801290F311DA901440FE5
:10437000551F240F351F245C3C4F869590E04C81DF
:10438000081719071CF4442331F002C0411103C07F
:1043900040913A0301C040E06091390380913803B5
:1043A0000E94C11D0F5F1F4FD5CF0E94401E8C8100
:1043B00090E00196817099278C83DF91CF911F91B6
:1043C0000F910895E7E3F3E080818E7F8083608121
:1043D0007181828193810E94E61D1092C0022FEFAD
:1043E00080E792E0215080409040E1F700C000005B
:1043F0000C94401E60913703669570E04BE050E0EE
:1044000084E191E00E949F34892B19F481E080932C
:10441000C0020E949B2C9093B9028093B802089529
:104420009091370390FF35C09170811102C0926066
:1044300006C0853210F0986402C0880F982B9093C4
:104440003703662351F060913703709138038091F0
:10445000390390913A030E94E61D609137036695F7
:1044600070E04BE050E084E191E00E949F34892BA2
:1044700019F01092C00202C00E94FA2181E08093DC
:10448000BB0240913A0360913903809138030C9448
:10449000E41F0895682F90913703969581E0890F66
:1044A000853208F081E00C94102281E00C944A22BD
:1044B000682F9091370396958FEF890F09F484E266
:1044C0000C94102281E00C94582261E00C9410228C
:1044D000E7E3F3E080818160808386950C94652218
:1044E0008091370380FD0C94E2210C94682260E0F7
:1044F0000C9410228091BE0281112EC00E9445159D
:10450000811104C00E94F2150E94F81D0E94E21D54
:1045100060933703709338038093390390933A0381
:104520006E7F61F40E94F81D0E94E21D60933703C4
:10453000709338038093390390933A030E94CF1D00
:104540001092C0028091370380FF03C086950E94BD
:10455000772281E08093BE0208950F931F93CF933B
:10456000DF938091C002882309F485C08091BF0247
:10457000E0913703E695E81BE093BA02823049F4F4
:10458000F0E0E952FA4FE491CE2FD0E009E91EE1C4
:1045900049C0863049F4F0E0EC52FA4FE491CE2F56
:1045A000D0E00DEA1EE13EC0893051F4E695F0E01E
:1045B000EF52FA4FE491CE2FD0E007EE1FE132C068
:1045C0008F3051F4E695F0E0E253FA4FE491CE2FAC
:1045D000D0E002E210E226C0853149F4F0E0E55374
:1045E000FA4FE491CE2FD0E00EE910E21BC08831E3
:1045F00081F0833239F4E9ECF5E0C591D4910DEB0B
:104600001EE110C0843251F4C4EFD1E003EA11E29C
:1046100009C0C8E2D0E000E111E204C0C0EDD7E07B
:104620000DEB1DE18091BB02882361F01092BB026B
:104630000E949B2C9093B9028093B8021092BD0205
:104640001092BC020E949B2CE091B802F091B9023A
:104650008E1B9F0B8F3F9F4770F4EC0FFD1FF09355
:10466000B902E093B80288EB92E0F801DF91CF91B4
:104670001F910F910994DF91CF911F910F91089590
:10468000882311F0FA0101C0FB010994CF93DF9355
:10469000C82FD62F0E94071E8C1740F00E94071EBD
:1046A0008D1720F4DF91CF910C9455228C2FDF9140
:1046B000CF910C9465221F93CF93DF93FB0112815E
:1046C0001111C3C0EC010E945C148272CD3CFCE568
:1046D000DF0709F49AC0A8F5C73CECE5DE0709F44A
:1046E00076C0A8F4C43C9CE5D90709F45FC028F45F
:1046F000C33CDC4509F457C054C0C53C9CE5D90710
:1047000009F459C0C63CDC4509F45CC04AC0CA3C47
:10471000FCE5DF0709F46AC050F4C83CECE5DE07AD
:1047200009F45AC0C93CDC4509F45BC03AC0CB3C33
:104730009CE5D90709F45FC0CC3CDC4509F460C0B6
:1047400030C0C23DFCE5DF0709F46FC088F4CF3C00
:104750009CE5D90709F460C008F45CC0C03DFCE5E5
:10476000DF0709F45CC0C13DDC4509F45BC019C03A
:10477000C53D9CE5D90709F460C050F4C33DFCE594
:10478000DF0709F455C0C43DDC4509F454C009C035
:10479000C63D9CE5D90709F455C0CE35DD4509F481
:1047A00054C011E052C00E9470224FC042E652E253
:1047B00065E572E204C045E552E262E672E20E94FB
:1047C000402343C045EA5FE168E97FE1F8CF48E96B
:1047D0005FE165EA7FE1F3CF43EC5FE164EB7FE10A
:1047E000EECF44EB5FE163EC7FE1E9CF41EE5FE1C7
:1047F00062ED7FE1E4CF42ED5FE161EE7FE1DFCF8B
:104800004AE35EE163E27EE1DACF43E25EE16AE33E
:104810007EE1D5CF81E017C065E082E010C068E09E
:1048200086E00DC06EE089E00AC064E18FE007C059
:1048300067E185E104C088E106C062E289E10E9487
:10484000462303C083E20E946522812FDF91CF912E
:104850001F910895549A2BB12F7E3BB130614FB711
:10486000F894FC01CB01880F991F680F791F6E0F18
:104870007F1FE617F70789F0819198E03BB90000A8
:1048800000C087FF2BB9880F000000C000C000C027
:104890002BB900C09A9591F7ECCF4FBF8FE594E00C
:1048A0000197F1F700C000000895EF92FF920F9377
:1048B0001F93CF93DF93EC017B0164E670E088E700
:1048C0000E94CB298C01EC0EFD1ECE15DF0561F098
:1048D00017FD0AC0FE01849164E670E00E944C2A34
:1048E0008C012196892B89F30E94D02AC801DF917F
:1048F000CF911F910F91FF90EF9008950895E6E6F4
:10490000F3E080E092E0DF019C011D9221503040F5
:10491000E1F7F0936D05E0936C058FEF9FEF9093B7
:10492000ED028093EC0208950E947E070E947E248F
:104930008093E80280FD02C080E801C080E280939D
:10494000E7020E94C5296DE070E087EF97E00E94C2
:104950005524892B11F080E008958091E80263E0EE
:1049600070E081FD03C084EF97E002C081EF97E023
:104970000E945524892B79F76DE070E084EE97E072
:104980000E945524892B39F70E94A72CDC01CB010A
:10499000805A9541AF4FBF4F80936805909369054A
:1049A000A0936A05B0936B050E947F2481E08093F9
:1049B000EB028093EA021092E90208952091E70247
:1049C00036E0839FC0011124629F800D911D112448
:1049D000811522E0920714F080E090E08A599C4F04
:1049E00090936D0580936C05089520916C0530912E
:1049F0006D05205633404091E702642F70E0C901F5
:104A00000E941534481B463010F4240F311D211527
:104A100082E0380710F020E030E02A593C4F309314
:104A20006D0520936C050895CF93DF938A3011F4C0
:104A300081E003C08D3029F480E0DF91CF910C94A8
:104A40008A25C62F682F80916C0590916D0526E010
:104A5000FC01A1ECB2E001900D922A95E1F7603ED5
:104A600030F026E0FC0111922A95E9F70AC0F6E041
:104A70006F9FB00111246C5F774F46E050E00E94B9
:104A80009634C11135C0C0916C05D0916D0546E0DA
:104A900050E0BE0181EC92E00E94AC34892BB1F170
:104AA000C656D3409E0185E0369527958A95E1F755
:104AB00081E090E0AC0102C0440F551F2A95E2F757
:104AC0002091EC023091ED02242B352B259645E008
:104AD000D695C7954A95E1F702C0880F991FCA95E8
:104AE000E2F7822B932B9093ED028093EC020EC0A1
:104AF000E0916C05F0916D059F012A5F3F4F2E17E5
:104B00003F0709F2808180958193F9CFDF91CF91A2
:104B10000C94F524CF93E82F20916C0530916D050E
:104B2000265633404091E702642F70E0C9010E948D
:104B30001534481B842FEE2359F066E00E94FB33A6
:104B4000C82FC150B0F060E080E20E941425F9CF78
:104B5000A901480F511D4115524018F080E020E096
:104B600030E0280F311D2A593C4F30936D052093BA
:104B70006C05CF9108953091E7028317C8F590E056
:104B8000262F269526952695239F800D911D11246D
:104B9000811522E0920764F5FC01EA59FC4F50812F
:104BA000677021E030E001C0220F6A95EAF74423E4
:104BB00011F0252B02C0209525232517C9F020834D
:104BC00025E0969587952A95E1F721E030E0A90147
:104BD00002C0440F551F8A95E2F7CA012091EC02EA
:104BE0003091ED02822B932B9093ED028093EC0297
:104BF00008951F93CF93DF93EC01162FFE0184914C
:104C0000882329F0612F0E9414252196F7CFDF9188
:104C1000CF911F9108958091EB028823F9F00E94B3
:104C2000A72CDC01CB01805A9541AF4FBF4F809339
:104C3000680590936905A0936A05B0936B05809110
:104C4000EA0281110BC062E070E082EE97E00E9400
:104C50005524892B19F481E08093EA028091EA02BD
:104C600008956F927F928F929F92AF92BF92CF9250
:104C7000DF92EF92FF920F931F93CF93DF93809178
:104C8000EB02882309F4DCC02091EC023091ED02A4
:104C90002115310509F4D4C08091E9028111D0C0F9
:104CA00061E070E0082F10E03B01082E02C0660CA6
:104CB000771C0A94E2F7A90146215721452B11F4EC
:104CC0008F5FF0CF9091E802980165E0220F331FCB
:104CD0006A95E1F790FD12C08295880F80768093E7
:104CE0002101220F232F221F330B31952093240102
:104CF000815E809322011092250112C045E0369515
:104D000027954A95E1F7220F220F220F20932101C8
:104D100010922401295F2093220183E080932501D2
:104D200024E630E047E050E06FE171E088E70E9460
:104D30007C2A892B09F084C08091E80280FD23C081
:104D4000A80195E0440F551F9A95E1F74A595C4F29
:104D500004E610E020E230E060E488E70E94A32A45
:104D6000892B09F06DC00E940B26E301C095D095F8
:104D70008091EC029091ED02C823D923D093ED02EB
:104D8000C093EC025DC080E2E7ECF2E0DF011D922F
:104D90008A95E9F785E0000F111F8A95E1F7A2EDEA
:104DA000B1E04EEC51E0992493942D91EA01899160
:104DB000AE01B801680F711D6A597C4F30E029536C
:104DC0003D4FF90197E07F01E21AF30AA92C01C0D7
:104DD000AA0CEA94EAF77B01B12CE70189917E01E4
:104DE0008A21892E8B18D82DD770CD2E0D2E000C30
:104DF000DD08C82F01C0CC0FDA95EAF7D194C19431
:104E0000D108D7E0CD22DD2401C08695CA94EAF707
:104E10008C2BD0808D298083B39488E0B812DDCFAD
:104E2000915031969F3F79F6C1E0A63DBC0709F04D
:104E3000BCCF04E610E020E230E047EC52E08CCF3B
:104E4000DF91CF911F910F91FF90EF90DF90CF9066
:104E5000BF90AF909F908F907F906F9008958091BA
:104E6000EB029091EA02882389F0992369F062E0CD
:104E700070E080EE97E00E945524892B19F0809114
:104E8000EA0208951092EA029091EA0281E08927ED
:104E9000089581E008950F931F938091EB0288237A
:104EA00099F180916605909167050E94B32C8197D6
:104EB00060F00E949B2C909367058093660560E0EC
:104EC00080E00E94DE240E9480070E9431268091AB
:104ED000EA028823C9F00E94A72C0091680510916E
:104EE000690520916A0530916B05DC01CB01801BBF
:104EF000910BA20BB30B8F3F9F4FAF4FBF4720F4D7
:104F00001F910F910C942F271F910F910895CF930C
:104F1000DF93EC01FB018281882309F43CC1C4309A
:104F2000FDE5DF0760F4CB3F9CE5D90788F49E01DF
:104F300022503C452431310508F02EC109C0C2364B
:104F4000EDE5DE0729F0C63AFDE5DF0709F024C1EB
:104F50000E945D159093220380932103C1318CE55B
:104F6000D80709F4C6C008F042C0C930ECE5DE0736
:104F700009F49BC000F5C5308CE5D80709F485C05D
:104F800078F4C330ECE5DE0709F478C008F07AC0A5
:104F9000C230DC4509F0F5C0809121038160EFC08B
:104FA000C7309CE5D90709F478C008F07AC0809131
:104FB00021038061E4C0CD30FCE5DF0709F487C040
:104FC00058F4CB309CE5D90709F479C008F07BC0D0
:104FD0008091210388606FC0CF30FCE5DF0709F4C2
:104FE00080C008F082C080912103877FC8C0CE3F77
:104FF0009CE5D90709F471C000F5C531FCE5DF0770
:1050000009F485C068F4C3319CE5D90709F475C07B
:1050100008F095C00E94E90E809121038F77AFC000
:10502000CC3FFCE5DF07A9F108F054C0CB3FDC45DD
:1050300009F0A7C08091220340C0C230EDE5DE0731
:1050400009F489C058F4C1158DE5D80709F45AC090
:1050500008F069C08091220382602FC0C236EDE55E
:10506000DE0709F47CC0C63AFDE5DF0709F481C01C
:10507000C330DD4509F085C080E06EC0809121031A
:1050800082607DC08091210316C0809121038860D9
:1050900076C08091220382604FC08091210380629C
:1050A0006EC08091210380646AC00E94E90E8091E5
:1050B0002103806864C0846062C081603DC08091CB
:1050C00021038E7F5CC0809121038D7F58C0809129
:1050D000210316C08091220318C0809122038D7F86
:1050E0002BC0809121038F7E4AC0809121038F7D48
:1050F00046C0809121038F7B42C080912103877F2E
:105100008B7F3DC0809122038D7F8E7F15C0809163
:10511000210382FB222720F991E0922790FB82F95C
:1051200090FB83F92CC080912203982F9095917069
:105130008E7F892B90FB81F98093220322C00E94ED
:10514000E90E8091210387FB222720F991E0922725
:1051500090FB87F914C081E00E94F41512C0809181
:10516000210384FB222720F991E0922790FB84F908
:1051700006C080912103982F909590FB80F9809331
:10518000210380912103909122030E946E150E94B9
:10519000E90E80E001C081E0DF91CF910895CF93C7
:1051A000DF9386319C4541F5EB010E945C14982FFA
:1051B0008A812091020130910301882379F09A7A43
:1051C00081E009F480E08093EE02911102C069E26F
:1051D00001C065E3C9010E94D72B0AC08091EE028D
:1051E000811102C069E201C065E3C9010E94E22B9E
:1051F0000E949E1480E001C081E0DF91CF9108956C
:105200000F931F93CF93DF93C42FD22FFC01828182
:105210008823C9F04093F1020E949B2C9093F002E6
:105220008093EF0280E28C0F883008F057C0C7707F
:1052300081E001C0880FCA95EAF7DF91CF911F91F5
:105240000F910C94460C8091F102481330C080916C
:10525000EF029091F0020E94B32C883C910538F542
:1052600010E21D0FCD17B9F080E28C0F883040F4AA
:10527000C77081E001C0880FCA95EAF70E944D0C03
:10528000183028F581E09D2F977001C0880F9A95FE
:10529000EAF70E94460C802F0E943D0C1830F0F473
:1052A000D77081E001C0880FDA95EAF70AC080E282
:1052B0008C0F883098F4C77081E001C0880FCA95C0
:1052C000EAF7DF91CF911F910F910C944D0C802F35
:1052D000DF91CF911F910F910C943D0CDF91CF91F5
:1052E0001F910F9108950F939C01CB01243F4CE532
:1052F000340731F188F4293DFCE53F07D9F02A3D18
:105300004CE5340779F1283D3C45A9F506E221EE4C
:1053100041EE68ED7CE52BC0263FFCE53F07E1F060
:10532000A8F0273F3C4539F507E225EE46EE67EF4A
:105330007CE51DC007E225EE45EE69ED7CE517C072
:1053400006E221EE40EE64EF7CE511C007E225EEB7
:1053500044EE65EF7CE50BC006E221EE42EE66EF1F
:105360007CE505C008E221E045EE6AED7CE50E949F
:10537000002980E008C0FC018281882319F0109286
:10538000F10201C081E00F9108951092B9008CE004
:105390008093B80008959F92AF92BF92CF92DF9210
:1053A000EF92FF920F931F93CF93DF93B82EEB01F1
:1053B0000E949B2C6C01C431D10558F0CF3F8FEF78
:1053C000D80759F0CE0164E170E00E9415347B01EA
:1053D00007C0EE24E394F12C03C025E0E22EF12C6B
:1053E00084E8A82E94EA992E1092BC009092BC00FA
:1053F0000E949B2C8C018091BC0087FD08C00E94FC
:105400009B2C801B910B8E159F05A8F32AC08091C1
:10541000B900887F883041F08091B900887F803161
:1054200019F00FEF1FEF1FC0B092BB00A092BC009D
:105430000E949B2C8C018091BC0087FD08C00E94BB
:105440009B2C801B910B8E159F05A8F30AC08091A1
:10545000B900887F883111F0803419F700E010E03E
:105460000EC00EEF1FEFCF3F8FEFD80709F4BCCF70
:10547000C6010E94B32C8C179D0708F4B5CFC80154
:10548000DF91CF911F910F91FF90EF90DF90CF9020
:10549000BF90AF909F9008950F931F93CF93DF938A
:1054A000EB018093BB0084E88093BC000E949B2C9E
:1054B0008C018091BC0087FD0EC0CF3F8FEFD807D5
:1054C000C1F30E949B2C801B910B8C179D0788F3C6
:1054D0008EEF9FEF0CC02091B900287F81E090E013
:1054E000283211F480E090E0919581959109DF9147
:1054F000CF911F910F910895CF92DF92EF92FF927B
:105500000F931F93CF93DF936B018A017901B90148
:105510000E94CB29E6010C0D1D1DC017D10761F4B7
:1055200024E92093BC00DF91CF911F910F91FF9050
:10553000EF90DF90CF90089597FDF2CFB70189915A
:105540000E944C2AEACFCF92DF92EF92FF920F9304
:105550001F93CF93DF93C62F6A017901B8010E9490
:10556000CB2997FD11C0B8018C2F0E944C2AE6016F
:10557000EC0CFD1CCE15DF0539F097FD05C0B80118
:1055800089910E944C2AF6CF24E92093BC00DF9138
:10559000CF911F910F91FF90EF90DF90CF900895E2
:1055A00084E98093BC0008959093D7018093D6013D
:1055B00008959093F7028093F6020895E091F60221
:1055C000F091F702309721F00190F081E02D0994DD
:1055D00080E008950E94DE2A0895E091F602F0919D
:1055E000F702309799F020913201222359F020914F
:1055F000210327FF07C0DC012C9111962C931197F2
:1056000026E02C930280F381E02D09940895E09127
:10561000F602F091F702309739F022E0DC012C938A
:105620000480F581E02D099408952091F4023091D1
:10563000F5022817390771F09093F5028093F40270
:10564000E091F602F091F702309721F00680F781A1
:10565000E02D099408952091F2023091F302281769
:10566000390771F09093F3028093F202E091F60211
:10567000F091F702309721F00084F185E02D099434
:105680000895FC01329680913201882331F0809197
:10569000210387FF02C09EE101C096E080E09150A7
:1056A00028F021912223D9F38F5FF9CF0895662343
:1056B00051F1209132012223E9F02091210327FFAB
:1056C00019C0462F4695469546954E31E0F46770D1
:1056D00021E030E002C0220F331F6A95E2F7FC019F
:1056E000E40FF11D828190E02823392381E0232BF0
:1056F00069F409C0FC01329608962191621729F0DD
:10570000E817F907D1F780E0089581E008959C013A
:10571000FC0132969FEF80E04191461789F09F3F50
:1057200019F4411101C0982F8F5F8630A9F79F3F70
:1057300039F0F901E90FF11D97FDFA95628308959B
:1057400008959C012A5F3F4FFC014281461301C02E
:105750001282019682179307B9F70895262F26958E
:10576000269526952E3168F4FC01E20FF11D677035
:1057700021E030E001C0220F6A95EAF78281282BF0
:1057800022830895262F2695269526952E3170F48E
:10579000FC01E20FF11D677021E030E001C0220F33
:1057A0006A95EAF720958281282322830895209123
:1057B0003201222329F02091210327FD0C94AE2BE6
:1057C0000C94872B20913201222329F02091210370
:1057D00027FD0C94C22B0C94A12B20913201FC01CB
:1057E0003296222331F08091210387FF02C08EE19F
:1057F00001C086E0DF011D928A95E9F708950895BA
:105800000C94FF2B83E08093F8020C94002C811100
:1058100002C081E001C082E08093F8020C94002C69
:105820000C94072C81E08093F8020C94002C0C94CB
:10583000122C08950C94192C0C941A2C0C94192CDD
:105840000C94192C0C94192CCF930E94202C0E949C
:10585000011A0E941E2CC0E08C2F0E942D19892B4A
:1058600029F4CF5FC530C1F780E001C081E0CF915E
:10587000089508951F920F920FB60F9211248F93DF
:105880009F93AF93BF938091F902811113C08091D0
:105890006E0590916F05A0917005B09171054196CC
:1058A000A11DB11D80936E0590936F05A0937005A7
:1058B000B0937105BF91AF919F918F910F900FBEE3
:1058C0000F901F90189580917605843031F10E94D9
:1058D000F9091092F90220E488E190E00FB6F894FB
:1058E000A895809360000FBE2093600083B7817FEE
:1058F000846083BF83B7816083BF7894889583B7C2
:105900008E7F83BF0FB6F894A89580916000886160
:1059100080936000109260000FBE08950E94E90E0F
:105920000C94FF0982E084BD93E095BD9AEF97BD8A
:1059300080936E0008952FB7F89480916E05909132
:105940006F05A0917005B09171052FBF08952FB715
:10595000F89460916E0570916F058091700590913B
:1059600071052FBF08959C014FB7F89480916E0583
:1059700090916F05A0917005B09171054FBF821B8A
:10598000930B089578941F920F920FB60F921124E3
:105990008F939F93AF93BF9380916E0590916F0506
:1059A000A0917005B09171050196A11DB11D809364
:1059B0006E0590936F05A0937005B0937105BF912C
:1059C000AF919F918F910F900FBE0F901F901895E0
:1059D000F89481E08093E00080E28093D800E9ECC5
:1059E000F0E010828FE19EE40197F1F700C0000023
:1059F0001DBA109268001CBC10BE1FBA10927A002B
:105A000010926E0010926F0010927100109272004E
:105A10001082ECEBF0E0108214B817B81AB81DB879
:105A200010BA108215B818B81BB81EB811BA0C9469
:105A3000003F089580911D030895089522E020936A
:105A4000E9002FEF3091E800215035FD06C035ED1B
:105A50003A95F1F700002111F5CF2091E80025FFDC
:105A60000BC040E050E066E070E00E945D2F809146
:105A7000E8008E778093E8000895CF93DF9320911C
:105A80003201222339F02091210327FF03C060E275
:105A900022E002C068E021E02093E9002FEF30917E
:105AA000E800215035FD06C035ED3A95F1F70000CC
:105AB0002111F5CF2091E80025FF1DC0EC01809158
:105AC0003201811105C040E050E068E070E003C0A1
:105AD00070E040E050E0CE010E945D2F8091E80030
:105AE0008E778093E80080E2FE01ADEFB2E0019096
:105AF0000D928A95E1F7DF91CF9108958093FA0294
:105B00007093FC026093FB0280917605843001F56E
:105B100082E08093E9008FEF9091E800815095FD3D
:105B200006C095ED9A95F1F700008111F5CF8091AF
:105B3000E80085FF0DC040E050E063E070E08AEFD0
:105B400092E00E945D2F8091E8008E778093E800BC
:105B50000895BC0184E00C947E2DBC0183E00C947C
:105B60007E2D80917505811109C00E94EE300E9442
:105B70004B318091E20084608093E200089510929E
:105B8000750508950C94172C6091720581E06111E0
:105B900001C080E00C94022C9091760581E0943055
:105BA00009F080E0609172050C94072C42E061ECF2
:105BB00081E00E94673042E261EC82E00E9467303F
:105BC0009091760581E0943009F080E06091720553
:105BD0000C94102C80917805833009F461C030F466
:105BE000813071F0823009F49AC008958A3009F446
:105BF00086C08B3009F46CC0893009F0A8C020C081
:105C000080917705813A09F0A2C08091E800877FF2
:105C10008093E80080917B0590917C05892B21F48D
:105C200060E28DEF92E003C060E080E090E070E021
:105C30000E94A82F8091E8008B778093E800089558
:105C400080917705813209F082C080917B05909127
:105C50007C05029708F07BC08091E800877F8093E5
:105C6000E8008091E80082FD05C0809176058111F1
:105C7000F8CF6DC02091F3008091F20090E0922B5C
:105C8000029731F48091F100813011F0863021F4D7
:105C90008091F10080931D038091E8008B7753C0C1
:105CA00080917705813A09F052C080917B059091EF
:105CB0007C05892B09F04BC08091E800877F809399
:105CC000E8008091E80080FFFCCF8091320136C06F
:105CD000809177058132D9F580917B0590917C0583
:105CE000892BA9F58091E800877F8093E8000E94C6
:105CF0009C3080917905809332010C94E90E80915B
:105D00007705813221F58091E800877F8093E80054
:105D10000E949C3080917A0580931E0308958091A3
:105D20007705813AA1F48091E800877F8093E800AD
:105D30008091E80080FFFCCF80911E038093F100EA
:105D40008091E8008E778093E8000C949C30089551
:105D500084B7877F84BF0FB6F894A89580916000C0
:105D6000886180936000109260000FBE90E080E830
:105D70000FB6F89480936100909361000FBE0C946D
:105D8000122C0E94EE300E944B31E2EEF0E0808156
:105D90008460808378940C94E03386E291E00C94E4
:105DA000D92A809176058530A9F4809176058530D1
:105DB00079F40E94632C809174058823B1F30E94CA
:105DC000242C882391F30E94472F0E94E90EEDCFE7
:105DD0000C948E2C089508950C94EE2E292F3327C1
:105DE00023303105C9F060F42130310581F02230D3
:105DF000310509F044C08BE390E02AE73DE043C061
:105E000021323105E1F02232310549F138C082E119
:105E100090E025EB3DE037C099278130910549F0AE
:105E200028F0029761F5E4E4FDE005C0E6E7FDE057
:105E300002C0E6E6FDE0849190E09F0124C0611578
:105E4000710541F061307105D1F489E090E025EAF7
:105E50003DE019C089E090E02CE83DE014C06115F8
:105E6000710541F06130710551F486EB90E027EC4B
:105E70003DE009C080E490E02DE73EE004C080E012
:105E800090E020E030E0FA0131832083089580E142
:105E900089BD82E189BD09B400FEFDCF8091D800A3
:105EA0008F7D8093D8008091E00082608093E00035
:105EB0008091E00081FDFCCF0895CF92DF92EF92B8
:105EC000FF920F931F93CF93DF93EC018B017A0125
:105ED0000E94BB30811133C0E114F10439F0F701A5
:105EE00080819181081B190BC80FD91FC12CD12C9F
:105EF0000115110519F18091E80085FD16C080910A
:105F0000E8008E778093E800E114F10449F0F7018E
:105F100080819181C80ED91ED182C08285E00FC0D8
:105F20000E94BB30882321F30AC089918093F1003D
:105F300001501109FFEFCF1ADF0ADACF80E0DF91BD
:105F4000CF911F910F91FF90EF90DF90CF90089528
:105F500020917D0530917E052617370748F06115A1
:105F6000710539F42091E8002E772093E80001C0F4
:105F7000B901FC0120E06115710579F18091760588
:105F80008823F1F18530F1F18091E80083FD3CC078
:105F90008091E80082FD2EC08091E80080FFEBCF69
:105FA0002091F3008091F20090E0922B6115710531
:105FB00051F08830910538F421912093F10061501F
:105FC00071090196F3CF21E0089709F020E0809154
:105FD000E8008E778093E800CECF2111CFCF0AC0A2
:105FE00080917605882361F0853061F08091E8002A
:105FF00083FD0AC08091E80082FFF2CF80E008951F
:1060000082E0089583E0089581E0089520917D0560
:1060100030917E052617370748F06115710539F470
:106020002091E8002E772093E80001C0B901FC011F
:1060300020E06115710591F180917605882309F4BE
:1060400040C0853009F43FC08091E80083FD3DC029
:106050008091E80082FD2FC08091E80080FFE9CFA9
:106060002091F3008091F20090E0922B6115710570
:1060700059F08830910540F424912093F100319635
:10608000615071090196F2CF21E0089709F020E0F4
:106090008091E8008E778093E800CBCF2111CCCFA0
:1060A0000AC080917605882361F0853061F0809187
:1060B000E80083FD0AC08091E80082FFF2CF80E013
:1060C000089582E0089583E0089581E00895982F6F
:1060D000973068F59093E900981739F07091EC00CB
:1060E0002091ED005091F00003C0242F762F50E056
:1060F00021FD02C09F5FECCF3091EB003E7F3093DB
:10610000EB003091ED003D7F3093ED003091EB00DE
:1061100031603093EB007093EC002093ED005093CE
:10612000F0002091EE0027FDE5CF80E008958F700C
:106130008093E90081E008958091770587FF11C081
:106140008091E80082FD05C0809176058111F8CF2D
:1061500011C08091E8008B770BC080917605882371
:1061600049F08091E80080FFF8CF8091E8008E77B9
:106170008093E80008952091E4003091E50095E6D1
:106180004091EC00842F817040FF23C08091E80093
:1061900080FD1DC080917605882399F0853099F0A7
:1061A0008091EB0085FD11C04091E4005091E50025
:1061B0002417350729F3915011F09A01E1CF84E0BB
:1061C000089582E0089583E0089581E0089580E0D5
:1061D00008954091E80042FFDDCF08950E945C31B0
:1061E0000E946431E0EEF0E0808181608083E8ED20
:1061F000F0E080818F77808319BCA7EDB0E08C91AF
:106200008E7F8C9380818F7E808310927505089598
:106210000F931F93CF93DF930E945C310E946431F0
:10622000C8EDD0E088818F778883888180688883F3
:1062300088818F7D888319BC109276051092720533
:10624000109274051092730500EE10E0F801808141
:106250008B7F808388818160888342E060E080E07A
:106260000E946730E1EEF0E080818E7F8083E2EE75
:10627000F0E0808181608083808188608083F80184
:1062800080818E7F8083888180618883DF91CF9138
:106290001F910F910895E8EDF0E080818F7E80835B
:1062A000E7EDF0E080818160808384E082BF81E05F
:1062B000809375050C940831E8EDF0E080818E7FC5
:1062C00080831092E20008951092DA001092E100AB
:1062D00008951F920F920FB60F9211242F933F93A0
:1062E0004F935F936F937F938F939F93AF93BF93DE
:1062F000EF93FF938091E10082FF0BC08091E20059
:1063000082FF07C08091E1008B7F8093E1000E94B3
:10631000DF338091DA0080FF1FC08091D80080FFBA
:106320001BC08091DA008E7F8093DA008091D900C3
:1063300080FF0DC080E189BD82E189BD09B400FE06
:10634000FDCF81E0809376050E94B12D05C019BC78
:10635000109276050E94BF2D8091E10080FF19C048
:106360008091E20080FF15C08091E2008E7F8093D3
:10637000E2008091E20080618093E2008091D80089
:1063800080628093D80019BC85E0809376050E94D6
:10639000C42D8091E10084FF30C08091E20084FF31
:1063A0002CC080E189BD82E189BD09B400FEFDCF2A
:1063B0008091D8008F7D8093D8008091E1008F7EFE
:1063C0008093E1008091E2008F7E8093E2008091D3
:1063D000E20081608093E20080917205882311F0D1
:1063E00084E007C08091E30087FD02C081E001C026
:1063F00083E0809376050E94CC2D8091E10083FF9D
:1064000029C08091E20083FF25C08091E100877F51
:106410008093E10082E0809376051092720580916E
:10642000E1008E7F8093E1008091E2008E7F809377
:10643000E2008091E20080618093E20042E060E04F
:1064400080E00E9467308091F00088608093F000C7
:106450000E94C22DFF91EF91BF91AF919F918F91BB
:106460007F916F915F914F913F912F910F900FBE50
:106470000F901F9018951F920F920FB60F92112434
:106480002F933F934F935F936F937F938F939F933C
:10649000AF93BF93CF93DF93EF93FF93C091E90046
:1064A000CF708091EC00D82FD17080FDD0E8109291
:1064B000E9008091F000877F8093F00078940E943B
:1064C0007F321092E9008091F00088608093F000A4
:1064D000CD2BCF70C093E900FF91EF91DF91CF9169
:1064E000BF91AF919F918F917F916F915F914F91EC
:1064F0003F912F910F900FBE0F901F9018951F93F3
:10650000CF93DF93CDB7DEB7AA970FB6F894DEBF6F
:106510000FBECDBFE7E7F5E08091F100819325E064
:10652000EF37F207C9F70E94EA2D8091E80083FF58
:106530002EC18091770590917805492F50E04A301F
:10654000510508F024C1FA01EE59FF4F0C945F3455
:10655000803821F0823809F01AC108C08091730593
:1065600090917405992389F082600FC080917B051A
:106570008F70873008F00BC18093E9008091EB00A9
:1065800085FB882780F91092E9009091E800977FB9
:106590009093E8008093F1001092F100D1C0282F71
:1065A0002D7F09F0F4C0882319F0823061F0EFC02C
:1065B00080917905813009F0EAC0933009F080E0DC
:1065C000809374052EC08091790581112AC0809135
:1065D0007B058F702FEF280F263008F0D8C08093EE
:1065E000E9002091EB0020FF1CC0933021F4809142
:1065F000EB00806214C09091EB0090619093EB00EF
:1066000021E030E0A90102C0440F551F8A95E2F74E
:106610004093EA001092EA008091EB00886080933A
:10662000EB001092E9008091E800877F8093E800FA
:106630000E949C30ACC08111AAC0109179051F77CF
:106640008091E3008078812B8093E3008091E800C3
:10665000877F8093E8000E949C308091E80080FF53
:10666000FCCF8091E30080688093E300111102C0A9
:1066700082E001C083E08093760589C08058823033
:1066800008F085C08091790590917A058C3D53E0A2
:10669000950779F583E08A838AE289834FB7F89476
:1066A000DE01139620E03EE051E2E32FF0E050934C
:1066B0005700E49120FF03C0E295EF703F5FEF7059
:1066C0008E2F90E0EA3010F0C79601C0C0968D93EF
:1066D0009D932F5F243149F74FBF8091E800877F5A
:1066E0008093E8006AE270E0CE0101960E94A82F34
:1066F00016C060917B0570917C05AE014F5F5F4FC6
:106700000E94EC2EBC01892B09F441C09091E80055
:10671000977F9093E80089819A810E94063080914A
:10672000E8008B778093E80032C0803881F5809153
:10673000E800877F8093E800809172058093F100E4
:106740008091E8008E7772CF811121C08091790508
:1067500090917A0599270297D4F48091E800877F79
:106760008093E80080917905809372050E949C30A7
:1067700080917205811106C08091E30087FD02C0FF
:1067800081E001C084E0809376050E94D62D80913F
:10679000E80083FF0AC08091E800877F8093E800CB
:1067A0008091EB0080628093EB00AA960FB6F8947C
:1067B000DEBF0FBECDBFDF91CF911F910895089529
:1067C000CF93809176058823A1F0C091E900CF7026
:1067D0009091EC00892F817090FD80E8C82B109279
:1067E000E9008091E80083FD0E947F32CF70C09362
:1067F000E900CF910895991B79E004C0991F96177D
:1068000008F0961B881F7A95C9F78095089587FB35
:10681000082E062687FD819567FD61950E94FB3352
:106820000EF4919507FC81950895AA1BBB1B51E1BD
:1068300007C0AA1FBB1FA617B70710F0A61BB70BF0
:10684000881F991F5A95A9F780959095BC01CD0195
:10685000089597FB072E16F4009407D077FD09D012
:106860000E94153407FC05D03EF4909581959F4F0A
:106870000895709561957F4F0895A1E21A2EAA1B85
:10688000BB1BFD010DC0AA1FBB1FEE1FFF1FA217E0
:10689000B307E407F50720F0A21BB30BE40BF50BDD
:1068A000661F771F881F991F1A9469F76095709566
:1068B000809590959B01AC01BD01CF010895EE0F2D
:1068C000FF1F0590F491E02D09940E946D3433234D
:1068D00012F48A1B9B0B0C947E34A29FB001B39FD1
:1068E000C001A39F700D811D1124911DB29F700DD9
:1068F000811D1124911D08950E946D34B7FF0895E4
:10690000821B930B08950E946D34A59F900DB49F38
:10691000900DA49F800D911D11240895B7FF0C9434
:1069200083340E948334821B930B0895FB01DC01A6
:1069300002C005900D9241505040D8F70895FC01D7
:106940004150504030F001900616D1F73197CF01F9
:106950000895882799270895FB01DC0104C08D91D3
:106960000190801921F441505040C8F7881B990BC1
:106970000895F999FECF92BD81BDF89A992780B507
:106980000895A6E1B0E044E050E00C94F334A8E1AF
:10699000B0E042E050E00C94F334262FF999FECF9A
:1069A00092BD81BDF89A019700B4021639F01FBA62
:1069B00020BD0FB6F894FA9AF99A0FBE089503967F
:1069C000272F0E94CE340E94CD34252F0E94CE3432
:1069D000242F0C94CE340196272F0E94CE340C9491
:1069E000CD34DC01CB01FC01F999FECF06C0F2BD2C
:1069F000E1BDF89A319600B40D9241505040B8F77D
:066A00000895F894FFCF99
:106A0600C8007002280850011E0A14010101020084
:106A16000E000E0E01191A1B1C1D1E1F202122001E
:106A260021007F2200031A2D3D2D1E2DAD2DA92DEF
:106A36001D2D01E200E900EA00B500B600B700CD61
:106A4600008301CC008A01920194012102230224D1
:106A5600022502260227022A02B300B4006F007044
:106A660000818283E200E900EA00B500B600B700C3
:106A7600CD008301CC008A019201940121022302F8
:106A860024022502260227022A02B300B4006F0060
:106A96007000818283F6F79667F5F4F1F09293958C
:106AA6003332313097C6343536000102020202060F
:106AB60006060909090909090F0F0F0F0F0F15150A
:106AC600151819191919191919191919232400084A
:066AD60010181810080062
:00000001FF
